:1080000000400020192D010029FF000029FF000079
:1080100029FF000029FF000029FF000000000000E8
:1080200000000000000000000000000029FF000028
:1080300029FF00000000000029FF0000F18500007A
:1080400029FF000029FF000029FF000029FF000090
:1080500029FF000029FF000029FF000029FF000080
:1080600029FF000029FF000029FF000029FF000070
:1080700029FF000029FF000029FF000029FF000060
:1080800029FF000029FF000029FF000029FF000050
:1080900029FF000029FF000029FF000029FF000040
:1080A00029FF000029FF000029FF000029FF000030
:1080B00029FF000029FF000029FF000029FF000020
:1080C00029FF000029FF000029FF000029FF000010
:1080D00029FF000029FF000029FF000029FF000000
:1080E00029FF000029FF000029FF000029FF0000F0
:1080F00029FF00000188000029FF000029FF00007F
:1081000029FF000029FF000029FF000029FF0000CF
:1081100029FF000029FF000029FF000029FF0000BF
:1081200029FF000029FF000029FF000029FF0000AF
:1081300029FF000029FF000029FF000029FF00009F
:1081400029FF000029FF000029FF000029FF00008F
:1081500029FF000029FF000029FF000029FF00007F
:1081600029FF00003911010029FF000029FF00004C
:1081700029FF000029FF000029FF000029FF00005F
:1081800029FF000029FF000029FF000029FF00004F
:1081900029FF000029FF000029FF0000E1FD000089
:1081A00029FF000029FF000029FF000029FF00002F
:0C81B00029FF000029FF000029FF00004B
:10840000FFFFFFFFFFFFFFFFFFFFFFFF7EF9FFFF03
:1084100010B5054C237833B9044B13B10448AFF3BE
:1084200000800123237010BD00C6FF1F0000000064
:10843000743101000C4B43B10C480D4910B5AFF33A
:1084400000800C48036823B910BD0A48036833B99B
:108450007047094B002BF7D0BDE810401847064B7A
:10846000002BF5D0184700BF000000007431010058
:1084700004C6FF1F74C5FF1F0000000080F31188B1
:1084800070472F4B41F238015A5842F478525A50F3
:108490002C4A927902F00C020C2A4FD041F244028D
:1084A0002949995003F558339A78110748BF9A78AB
:1084B000264944BF42F008029A70214B41F244021F
:1084C000995041F204015A5842F4803242F0C002FD
:1084D0005A501A6842F440221A6003F5E833242205
:1084E0005A701B4A80211170A2221A70DA7802F0A9
:1084F0001F02DA7007221A710C225A719A799207B8
:10850000FCD59A79D006FCD40E4B19469A7902F024
:108510000C02082AFAD14C225A718B7903F00C0311
:10852000082BFAD1074B1A4699794906FCD5222126
:108530001970937903F00C030C2BFAD1704700BF2C
:1085400000700440004006400000330100001301A9
:1085500000500640234B5A7902F0E0025A711A7912
:1085600002F0F8021A71A3F500531A7802F08C0297
:1085700042F050021A705A7802F09C0242F0400217
:108580005A709A7802F0E6029A70174A0023137024
:1085900083F31188154B012283F8182383F81923DC
:1085A000022283F8582383F8592383F81D2383F884
:1085B0001E2383F81F2383F8202383F8212303221B
:1085C00083F82D2383F82F2383F8312383F8332373
:1085D00083F83523042283F85723052283F849239F
:1085E000704700BF00F0074000E0074000E100E0F6
:1085F000314A13680133F0B51360304A1368013310
:1086000013602F4B1A683AB11A68013A1A601B6856
:1086100013B92C4B01221A702B4B1A6812B11A682D
:10862000013A1A60294B5A68294B92B21A60294ABA
:1086300018681168884223DD19681068264C091AE9
:10864000B1F5004F25480ADA1E6817682168D0E99D
:108650000045F61B7143641845EBE1750BE01968A2
:1086600017682668D0E90045C91BC1F58031714300
:10867000641A65EBE175C0E900451B681360F0BD45
:10868000186811688842F8DA11681868124C091ADB
:10869000B1F5004F114806DA16681F682168F61B0D
:1086A000D0E90045E3E711681F682668C91BD0E9D7
:1086B0000045C1F58031CDE71CC6FF1F6CD0FF1F00
:1086C000FCCCFF1FF8CCFF1F00CDFF1F0090034024
:1086D0001CCDFF1F18CEFF1F58CDFF1F60CDFF1F01
:1086E00041F23C0205498B5843F000738B50044B18
:1086F000044A5A6007221A60704700BF00700440A5
:1087000010E000E040190100014B1868704700BFFD
:108710001CC6FF1F1449154B41F234020B2888BFB9
:10872000002010B553F82030114CB4FBF3F48B58F3
:1087300043F480638B500F4B4FF400725A602D202E
:108740009A6007F009FC0C4B0022DA709A709A715B
:10875000DA725A71C4F30422E4B21A705C70DA78E7
:1087600042F02C02DA7010BD00700440B42F0100FA
:1087700020AA44000090044000A00640094A136863
:1087800051680133202B08BF00238B4208D01168A9
:10879000114408721360044AD37843F08003D37005
:1087A000704700BF20C6FF1F00A006400A4B996A11
:1087B000DA6A91420DD09A6A511C1A44996292F871
:1087C000302002709A6A202A01D100229A62012088
:1087D00070470020704700BF20C6FF1F044B1A7867
:1087E00002F0FF0012B100221A700120704700BF92
:1087F000F8CCFF1F014B1865704700BF20C6FF1F54
:1088000030B526480179C9B28C0617D5244BDA6AEF
:108810009C6A0132202A08BF0022A2421BBFDC6AE8
:10882000C579C27918191EBFEDB280F83050DA62EE
:108830001C4A052010601A6D1B4B1A604A0608D5A9
:108840001A4B4FF400329A60144AD37803F0BF03F6
:10885000D3700B061BD5144B1868C0B9104B1968A0
:108860005A68914214D0114A4FF4003151605A684D
:10887000511C1A445960117A084AC9B2D171596819
:10888000202908BF5860D37843F04003D37030BD2F
:10889000024AD37803F07F03F8E700BF00A0064048
:1088A00020C6FF1FFCCCFF1F00CDFF1F00F00F40B4
:1088B00062B67047FFF7FCBF72B67047FFF7FCBFA8
:1088C0004FF0E02318B1034AC3F80C2D7047024A59
:1088D000FAE700BF0400FA050100FA0510B9C9085B
:1088E00001F0E6BC7047F7B5454A464E46494FF49D
:1088F0008073136153619363D36313645364716131
:10890000B160424940F20310086048608860C86066
:108910008862C8620B644B6401F5352140314FF425
:108920004030486148603A4840F6070403604360BD
:108930008360C3624C654C643649374C0B604B60B6
:108940008B60CC600B614B6101F53321C031142485
:108950004C6104244C6010248C60304C636104F53D
:10896000322404F580742025656141F204042C4D05
:108970002F5927F0E0072F512F5947F0C0072F51EB
:108980004FF4A064C46013603446D360082600230B
:108990000A201A46B4461F46A646C4F804C00197EA
:1089A000019DB5F57A7F21D3DEF81050A660ED0762
:1089B00048BF01320197019DB5F57A7F1AD3DEF8E1
:1089C0001050ED0758BF01330138E6D10A2A154A85
:1089D00014D10A2B12D101231370094B4FF4E0621A
:1089E0001A60DA6010234B6003B0F0BD019D0135C1
:1089F0000195D5E7019D01350195DCE70023EBE703
:108A00000090044000F00F402880030000A00440C4
:108A100000B0044000C004400001090000D0044040
:108A20000070044054CDFF1FF7B5114B1B78E3B124
:108A300010491148114D20231E4600240F4686463A
:108A40004E6086600194019AAA420AD9BB60CEF8B2
:108A500004300194019AAA42F2D8019A013201929B
:108A6000F8E7019A01320192EDE703B0F0BD00BFD3
:108A700054CDFF1F00F00F4000F10F401FA1070071
:108A8000072809D8DFE800F004090C0F11141618A4
:108A90004FF400420A4B5A6070474FF48032F9E7B6
:108AA0000222084BF7E70822FBE74FF40062F8E7E1
:108AB0000122F6E70422F4E74FF48062F1E700BFF9
:108AC00000F00F4040F00F40072809D8DFE800F021
:108AD00004090C0F111416184FF400420A4B9A6047
:108AE00070474FF48032F9E70222084BF7E708227B
:108AF000FBE74FF40062F8E70122F6E70422F4E70F
:108B00004FF48062F1E700BF00F00F4040F00F40EB
:108B100038B500210446012505FA01F32342C8B205
:108B200005D0FFF7ADFF01312029F5D138BDFFF7A2
:108B3000CBFFF8E708B506282CD8DFE800F0040DD5
:108B400012171C212600002006F090FFB0F5806F60
:108B500034BF0020012008BD0F4B186900F0010050
:108B600008BD0D4B1869C0F3800008BD0A4B186999
:108B7000C0F3802008BD084B1869C0F3400008BD51
:108B8000054B1869C0F3C00008BD034B1869C0F35A
:108B9000C02008BD002008BD40F00F4007282DD898
:108BA000DFE800F004090E13181D2227144B186883
:108BB000C0F3C0307047124B1868C0F300407047D4
:108BC000104B1868C0F3400070470E4B1868C0F394
:108BD000C00070470B4B1868C0F3C0207047094BAA
:108BE000186800F001007047064B1868C0F3800059
:108BF0007047044B1868C0F380207047002070470E
:108C000000F00F4040F00F4070B5002425460126CB
:108C1000E0B2FFF78FFF10B106FA04F31D430134F1
:108C20001F2CF5D1284670BD10F0010F314B33D009
:108C30005A6942F002025A614FF400329A6010F011
:108C4000020F2D4A30D0596941F0080159610221C3
:108C5000916041072FD5596941F4006159614FF482
:108C60000061916001072ED5596941F001015961F8
:108C70004FF480319960C1062DD5596941F0040146
:108C800059610121916081062CD5596941F48061B7
:108C900059610423936070474FF400325A605A6957
:108CA00022F002025A61CAE702215160596921F09B
:108CB00008015961CDE74FF400615160596921F411
:108CC00000615961CEE74FF480315960596921F054
:108CD00001015961CFE701215160596921F0040177
:108CE0005961D0E7042151605A6922F480625A61C7
:108CF000704700BF40F00F4080F00F401B4B5A6898
:108D000010F0010F14BF42F0030222F001025A607A
:108D1000DA6881074CBF42F0030222F00102DA60F8
:108D2000124BDA6A10F0040F14BF42F0030222F073
:108D30000102DA621A6801074CBF42F0030222F016
:108D400001021A60094B9A6810F0100F14BF42F02C
:108D5000030222F001029A609A6A81064CBF42F037
:108D6000030222F001029A62704700BF00A0044093
:108D700048B9064BD3F8A020120705D50822C3F83E
:108D8000A020012070470020704700BF00C00440B1
:108D900008B5082006F06AFE5E2810D9124B1A7832
:108DA0000AB901221A70082006F060FE63280ED965
:108DB0000E4B1B785BB90E4B04229A6008BD08204D
:108DC00006F054FE5428EED80022074BEAE70820AC
:108DD00006F04CFE542802D9044B1B7813B1044B07
:108DE00004225A6008BD00BF74C6FF1F3CCDFF1FA0
:108DF000C0F00F40034B1878013801288CBF0020C9
:108E00000120704774C6FF1F034B1878012806BF66
:108E100002221A700020704774C6FF1FC0B201F012
:108E200085BBC0B201F078BB08B508F0A9FF07F018
:108E300067FA07F017FABDE8084009F023B838B51B
:108E4000054607F065F908280AD9002428190134D5
:108E500007F0DEF9092CF9D107F00EFA012038BD30
:108E6000002038BD092107F073B9002007F000BCCD
:108E70002149224841F23C028B5843F440538B5025
:108E80001F4B012119601A6802431A601D4ADA60FB
:108E90001A61DA6A42F08052DA621A6822F001023C
:108EA0001A601A6822F000621A6003F5F8334FF472
:108EB00000721A615A619A61DA61A3F5F0331960A0
:108EC0001968014319601049D96001F52001196141
:108ED000D96A41F08051D962196821F00101196005
:108EE000196821F00061196003F500331A605A60B7
:108EF0009A60DA601A61704700700440000C1F80AD
:108F000000C002400300013E0400513EFF281ED86D
:108F100000041E4B00F47C108AB141F0006108434C
:108F20005863DA6A002AFCDA184BDA6AD100FCD5F9
:108F3000986BDA6A42F01042C0B2DA62704741F0D0
:108F4000004108435863DA6A002AFCDAF0E7B0F51A
:108F5000007F18D200040E4B00F47C105AB141F08F
:108F6000006108435863DA6A002AFCDA084BDA6ABF
:108F7000D200FCD5DCE741F0004108435863DA6ACF
:108F8000002AFCDAD4E70020704700BF00C002408E
:108F900000D00240C0EBC00038B500220C4600F5FE
:108FA000006503210120FFF7B1FF0022C5F307216F
:108FB0000120FFF7ABFF0022E9B20120FFF7A6FF77
:108FC000002211460120FFF7A1FF00221146207068
:108FD0000120FFF79BFF0022114660700120FFF780
:108FE00095FF00221146A0700120FFF78FFF00229D
:108FF0001146E0700120FFF789FF00221146207121
:109000000120FFF783FF0122607100211046FFF766
:109010007DFFA07138BD38B54FF4006401220621F0
:109020001046FFF773FF002205210120FFF76EFFB6
:10903000012200211046FFF769FF8007F3D50022C7
:1090400002210120FFF762FF0022C4F30721012063
:10905000FFF75CFF0022E1B20120FFF757FF002578
:10906000A5F13F014A424A41012000210135FFF7A5
:109070004DFF402DF4D1002205210120FFF746FFCE
:10908000012200211046FFF741FFC307F3D440340B
:10909000B4F5804FC2D138BDF7B5C0EBC00000F5C4
:1090A00000650C46002203210120FFF72FFFC5F3C6
:1090B000072100220120FFF729FFE9B20022012049
:1090C000FFF724FF002211460120FFF71FFF0022B7
:1090D000114607460120FFF719FF002211460646F8
:1090E0000120FFF713FF0022114605460120FFF77C
:1090F0000DFF002211468DF803000120FFF706FF47
:10910000002211468DF804000120FFF7FFFE012226
:109110008DF8050000211046FFF7F8FE23788DF842
:109120000600BB420ED16378B3420BD1A378AB42A9
:1091300008D1DDF80300D4F80330C31A584258416F
:1091400003B0F0BD0020FBE7012238B504460D4610
:1091500010460621FFF7DAFE002205210120FFF765
:10916000D5FE012210460021FFF7D0FE8207F3D57D
:10917000002202210120FFF7C9FE0022C4F30721CB
:109180000120FFF7C3FE0022E1B20120FFF7BEFE7F
:10919000012229461046FFF7B9FE002205210120D1
:1091A000FFF7B4FE012200211046FFF7AFFEC30710
:1091B000F3D438BD38B50D46C0EBC00404F50060EB
:1091C0000978FFF7C1FF697804F60100FFF7BCFFDB
:1091D000A97804F60200FFF7B7FFE97804F6030068
:1091E000FFF7B2FF297904F60400FFF7ADFF6979B4
:1091F00004F60500FFF7A8FFA97904F60600BDE80C
:109200003840FFF7A1BF2DE9F84316460122044676
:10921000884610460621FFF779FE0022052101202D
:10922000FFF774FE012200211046FFF76FFE85074D
:10923000F3D5002202210120FFF768FE0022C4F3CB
:1092400007210120FFF762FE0022E1B20120FFF7B3
:109250005DFE0025771EB5420DD1002205210120BB
:10926000FFF754FE012200211046FFF74FFEC3070F
:10927000F3D4BDE8F883013414F03F0918F8051061
:1092800039D0781B424242410120FFF73FFEB9F13D
:10929000000F2ED1BD422CD2002205210120FFF764
:1092A00035FE012200211046FFF730FEC107F3D43E
:1092B000012206211046FFF729FE00220521012088
:1092C000FFF724FE012210460021FFF71FFE820750
:1092D000F3D5002202210120FFF718FE0022C4F37B
:1092E00007210120FFF712FE0022E1B20120FFF763
:1092F0000DFE0135AFE70122C6E710B50022044696
:1093000003210120FFF702FEC4F307210022012000
:10931000FFF7FCFDE1B200220120FFF7F7FD01227B
:1093200000211046BDE81040FFF7F0BDF8B5044637
:109330000E461546032100220120FFF7E7FDC4F386
:10934000072100220120FFF7E1FDE1B20022012008
:10935000FFF7DCFD77193446013DBC4200D1F8BD72
:10936000A21BAB1A5A425A4100210120FFF7CEFD41
:1093700004F8010BF1E7F7B5002205210120FFF702
:10938000C5FD012200211046FFF7C0FD10F0710459
:10939000F2D1FFF7B9F90546FFF7B6F9401B0028EF
:1093A000B8BF4042B0F5FA6F22DAC4B1334B1B7834
:1093B00003BB402232490020FFF7B8FF2022314989
:1093C0004020FFF7B3FF20222F496020FFF7AEFFB8
:1093D00020222E498020FFF7A9FF03B0F0BD40F204
:1093E000FF70FFF78AFFA0F1AA035C425C41D3E75C
:1093F000002CDBD1002140F2FF70FFF7A5FEFFF744
:109400000AFE40221E49224F224E0020FFF7FBFE9B
:1094100040254FF480742046B4223946FFF7F3FE0E
:10942000B434284620223146FFF7EDFEB4F5477FDD
:1094300005F12005EFD102AD002345F8043D4FF4BE
:10944000C3642046042229460434FFF7DCFEB4F549
:10945000FF6FF6D1002301934FF4A7642046042246
:1094600029460434FFF7CFFEB4F5C36FF6D1AA2125
:1094700040F2FF70FFF768FE9BE700BF54CDFF1F6F
:109480000CC0FF1FB8CDFF1FD8CDFF1FF8CDFF1FA9
:1094900004300100E42F01002DE9F0411378C3F3FB
:1094A000411507460E46144615BB3D4A117BF9B9D6
:1094B000D8071DD45F2B1BD83A490978C1B913F0DE
:1094C000970F15D1DFF8E48098F800302BB1517A6E
:1094D0002846FFF703FA88F80050DFF8D48098F8A0
:1094E00000302BB1002001F021F8002388F8003073
:1094F0000022217840F20110FFF708FD30700022B1
:10950000617840F20110FFF701FD70700022A17830
:1095100040F20110FFF7FAFCB070E178012240F24E
:109520000110FFF7F3FCF0702378D90735D45F2BD7
:1095300033D803F01E03082B11D0142B24D0062B94
:109540002BD124237B430C2707FB0537164DA2782C
:10955000E3783D4443EA02236B60BDE8F081A278E2
:10956000E378114943EA0223242257430C2202FBE9
:1095700005754B51A27812070FD56FEA03536FEAB6
:1095800013534B51BDE8F08124235F430C2303FBAD
:109590000575054BE2781D442A72BDE8F08100BFD5
:1095A000B8CDFF1F74CEFF1F68CDFF1F71CEFF1F08
:1095B00077CEFF1F07B513788DF8013053788DF8FB
:1095C00000108DF8023001A993788DF803306A46B7
:1095D000FFF762FF03B05DF804FB07B58DF80010DC
:1095E0008DF801208DF802306A469DF810308DF814
:1095F000033001A9FFF750FF03B05DF804FB07B586
:1096000000238DF800108DF801308DF8032013121F
:1096100001A96A468DF80230FFF73EFF03B05DF8FE
:1096200004FB5F292DE9F34180460F46144606D816
:1096300017F01E064FEA511113D0022E2ED023141C
:109640008DF801306A46231201A940468DF800705A
:109650008DF802308DF80340FFF71EFF02B0BDE821
:10966000F081032212FB0012244B2548120103EB68
:10967000020E9C50DEF80410651A002DB8BF6D4232
:10968000854208DD13448C424FF00102CCBF0C1818
:109690000C1A1A73D3E78EF80C60D0E7032616FB7A
:1096A0000016164D3601AA1955F806E05460AEEBC7
:1096B000040024F07F4300289360114BB8BF404260
:1096C000984217DD7445B4BF1B19E31A4A018DF89F
:1096D00000201A148DF801201A128DF8022001A919
:1096E0006A46404635448DF80330FFF7D5FE012326
:1096F0002B73A4E700231373A1E700BFACCEFF1FB9
:10970000FFFF7F0007B511F01C0204D1FFF789FFAE
:1097100003B05DF804FB00238DF800106A4601A930
:109720008DF801308DF802308DF80330FFF7B4FE6C
:10973000EEE70122114640F20110FFF7E7BB13B537
:10974000144602AA41F0010102F8041D6946FFF720
:10975000A3FE9DF8013023709DF8023063709DF8E0
:1097600000009DF80330A37002B010BD07B502AA37
:1097700041F0010102F8041D6946FFF78DFEBDF8B6
:10978000020040BA80B2030544BF6FEA00506FEA9E
:10979000105003B05DF804FBF7B5490102AD4CB2BF
:1097A00044F0150305F8083D174601A92A46064668
:1097B000FFF772FE9DF805308DF8013044F0140477
:1097C0009DF806308DF800402A4601A930468DF8F4
:1097D00002308DF80370FFF75FFE03B0F0BDF7B500
:1097E000490102AD4CB244F0150305F8083D174697
:1097F00001A92A460646FFF74FFE9DF805308DF871
:10980000013044F014049DF807308DF800402A46DA
:1098100001A930468DF802708DF80330FFF73CFE49
:1098200003B0F0BD73B502AC7F2304F8083D0D46CC
:10983000224601A90646FFF72FFE7E238DF8003051
:109840009DF805308DF8013005F00F059DF80730C3
:109850008DF80250224601A930468DF80330FFF7FB
:109860001BFE02B070BD2DE9F74F400145B2C1F3B8
:109870000A0845F0180101AA01F0F8010020FFF7DD
:109880005EFF9DF805404FEA141904F00F04A1454E
:1098900040465CDC08F04CFCA4EB090406460120C1
:1098A000A0400F4608F054FC0022334B08F0B6FCF1
:1098B00002460B463046394608F0DAFD08F0E8FE6D
:1098C00008F058FC2AA3D3E9002308F0A7FC08F00D
:1098D000DFFE08F04FFC0022284B08F09FFC4FF001
:1098E000FF3906460F46CA4600244FF0010B0BFA1B
:1098F00004F008F02DFC3B46324608F08FFC08F0DF
:109900009FFEA0F180037F2B98BFA14604F10104C4
:1099100098BF82460E2CEAD1002445F0120101AA1C
:10992000204601F0F2018DF804408DF805A08DF875
:109930000690FFF73FFE45F00C012046424601F03D
:10994000EC01FFF75CFE204603B0BDE8F08F08F0A5
:10995000EFFBA9EB040406460120A0400F4608F0E7
:10996000F7FB02460B460020034908F081FD9FE704
:1099700004560E2DB29DEF3F0000604000002040D5
:1099800073B54A0803244FF4807314FB0233B424E4
:1099900014FB0034064620460D46FFF7AEFC8DF85A
:1099A0000400601CFFF7A9FC8DF80500A01CFFF760
:1099B000A4FC45EA46118DF8060001AAC9B20020B0
:1099C000FFF7F8FD02B070BD73B50D4641EA4011D6
:1099D00001AA0646C9B20020FFF7B1FE03244FF4E6
:1099E00080736D0814FB0535B42414FB06549DF8F0
:1099F00004102046FFF7A8FB9DF80510601CFFF738
:109A0000A3FB9DF80610A01CFFF79EFB02B070BDE3
:109A100010B5C4B221466401E4B202220020FFF76F
:109A2000BBFE44F008010020FFF76CFE44F00A0181
:109A30000020BDE81040FFF765BE37B5440144F093
:109A40001604E4B20D4601AA21460020FFF777FE76
:109A50009DF8053015F0010F14BF43F0400323F0CB
:109A600040038DF805309DF8053015F0020F14BF46
:109A700043F0100323F01003002001AA21468DF8C3
:109A800005308DF80600FFF795FD03B030BD37B502
:109A9000440144F01604E4B20D4601AA2146002018
:109AA000FFF74DFE9DF8053015F0010F14BF63F070
:109AB0007F0303F07F038DF805309DF8053015F026
:109AC000020F14BF43F0200323F02003002001AA5B
:109AD00021468DF805308DF80600FFF76BFD03B0C9
:109AE00030BD07B5410141F0160101AA01F0F601B0
:109AF0000020FFF724FE9DF80530C3F38010DB063D
:109B000048BF40F0020003B05DF804FB07B5410117
:109B100041F0160101AA01F0F6010020FFF70FFE47
:109B20009DF80530D8099B0648BF40F0020003B0FD
:109B30005DF804FB70B5104C05016219204693686E
:109B40008B420DDACB1AC3F18076B342546804DC41
:109B5000234453602844816070BDA41B5460F9E71E
:109B6000F8DD5B1AC3F18076B342546801DCE31A76
:109B7000EFE73444F2E700BFACCEFF1F73B502AA93
:109B800041F001030C4602F8043D69460546FFF723
:109B900083FC9DF802009DF80110000240EA01409C
:109BA0009DF803100843030248BF40F07F405F2C3C
:109BB00005D8660914F01E0403D0022C08D002B0A8
:109BC00070BD032010FB05600001094B1858F6E733
:109BD00005EB4503334420F07F41D8B2FFF7AAFFDD
:109BE000032010FB0560024D05EB00156868E6E7F1
:109BF000ACCEFF1F38B50D4668210446FFF7BEFF07
:109C00003DB140F0010220466821BDE83840FFF731
:109C100008BD20F00102F6E773B51C4B587E10F02A
:109C200001001DBF40F22312682100204FF4917201
:109C300008BF6821FFF7F5FC0223009300231A46B2
:109C40007E211846FFF7C9FC00240025E6B2E9B2E0
:109C500030460135FFF794FE1D2DF8D17501EDB2A8
:109C600045F00C010020FFF789FF01463046FFF761
:109C7000FAFD013443F2FF1245F016010020FFF710
:109C8000BEFC032CE1D102B070BD00BF0CC0FF1FB1
:109C90007FB5450104AA45F0030302F8043D0446DC
:109CA00002A90020FFF7F8FB9DF80A309DF8091083
:109CB0001B0243EA01439DF80B1020461943FFF7AE
:109CC00039FF134A2301D118087BE8B111480C264B
:109CD00006FB0404267ABEB9D2584B680E48D41A43
:109CE000002CB8BF6442844210DD9A42CCBF1A18DF
:109CF0001A1AD3B2009305F0E001C2F30723002043
:109D0000C2F30742FFF769FC04B070BD0E73F0E7C1
:109D1000ACCEFF1F68CDFF1FFFFF7F0038B5C0F33B
:109D20000741054600224FF48170FFF7EFF80C4C15
:109D3000000220600022C5F307214FF48170FFF775
:109D4000E5F823681843000220600122E9B24FF4CD
:109D50008170FFF7DBF8236818430009206038BDE5
:109D600078C6FF1F10B5244CC00023181A79032AA7
:109D700084BF03221A7123189A79032A84BF03220D
:109D80009A7123181A7A0F2A84BF0F221A72231885
:109D90005A7A072A84BF07225A7223189A7A0F2AFE
:109DA00084BF0F229A72221813795279DB0343F48D
:109DB0000021E16012B143F40423E3602318DB794E
:109DC0001BB1E36843F40053E3602044037A8279D3
:109DD000DB0143EAC223E2681343427A43EA0213F7
:109DE000C27AE36012B9827A1343E360E068FFF756
:109DF00095FFE368236110BD78C6FF1F10B5104CB6
:109E00000023C000E36023185B7E13B14FF400739E
:109E1000E36023189B7E1BB1E36843F48073E36027
:109E200023182044DA7E0F2A84BF0F22DA76C07E00
:109E3000E3681843E060FFF771FFE368E36110BD7A
:109E400078C6FF1F38B5C2001F4C111A214491F883
:109E5000213091F8205091F822101B0343EA8533FA
:109E600043F46025012908BF2B46A2EB000108BF7F
:109E700043F480632144E56008BFE360E36891F840
:109E8000235091F8241043EA05230129E36004BF1D
:109E900043F08003E360131A2344121A93F8253029
:109EA000012B08BFE368224404BF43F04003E36092
:109EB000E06892F8263040EA0310E060FFF72EFFDA
:109EC000E368A36238BD00BF78C6FF1F10B543002A
:109ED0001C4C1A18224492F92D103F29C4BF3F216F
:109EE00082F82D101A18224492F92D103F31BCBF70
:109EF000C12182F82D101A18224492F82E101F2921
:109F000084BF1F2182F82E104FF44022E2601A18FD
:109F10002244034492F82C202344012A04BF4FF426
:109F20005022E26093F82D00E26893F82E30000290
:109F3000134300F4FE401843E060FFF7EFFEE368D0
:109F4000236310BD78C6FF1F10B58300244C1A1878
:109F5000224492F83410012984BF012182F8341080
:109F60001A18224492F83510032984BF032182F87D
:109F700035101A18224492F836100F2984BF0F2189
:109F800082F836101A18224492F83710032984BF39
:109F9000032182F837101A182244034492F838102B
:109FA0000F29234484BF0F2182F8381093F838001A
:109FB00093F8342040F4202040EAC23093F8352052
:109FC00040EA423093F8362093F8373040EA0220D6
:109FD00040EA4310E060FFF7A1FEE368E36310BDD1
:109FE00078C6FF1F214B012010B503210024052254
:109FF00083F82C0083F825000220597283F8201082
:10A0000083F8211018729A72DC7283F82D2083F87D
:10A010002E2083F8224083F8234083F8244083F8DD
:10A02000260083F8344083F8354083F8364083F8BF
:10A03000374083F838405C769C76DC7618715C712A
:10A04000DC719C710A4B04229A602046FFF77CFF6A
:10A050002046FFF73BFF2046FFF7F4FE2046FFF7C0
:10A06000CDFE2046BDE810407CE600BF78C6FF1F4D
:10A07000C0F00F40044B042903EBC00318BF0022BB
:10A08000D97618BF5A76B9E678C6FF1F034B03EBA3
:10A09000C003597609B10422DA76AFE678C6FF1F0D
:10A0A000024B03EBC0039976A8E600BF78C6FF1FFA
:10A0B000024B03EBC000C07E704700BF78C6FF1F95
:10A0C000024B03EBC000407E704700BF78C6FF1F05
:10A0D000024B03EBC000807E704700BF78C6FF1FB5
:10A0E000024B03EBC00319713CE600BF78C6FF1FAB
:10A0F000024B03EBC003597134E600BF78C6FF1F63
:10A10000024B03EBC003D9712CE600BF78C6FF1FDA
:10A11000024B03EBC003997124E600BF78C6FF1F12
:10A12000024B03EBC00319721CE600BF78C6FF1F89
:10A13000024B03EBC003597214E600BF78C6FF1F41
:10A14000024B03EBC00399720CE600BF78C6FF1FF9
:10A15000024B03EBC0000079704700BF78C6FF1FB9
:10A16000024B03EBC0004079704700BF78C6FF1F69
:10A17000024B03EBC000C079704700BF78C6FF1FD9
:10A18000024B03EBC0008079704700BF78C6FF1F09
:10A19000024B03EBC000007A704700BF78C6FF1F78
:10A1A000024B03EBC000407A704700BF78C6FF1F28
:10A1B000024B03EBC000807A704700BF78C6FF1FD8
:10A1C000034B00EB8002134483F83410BCE600BF5D
:10A1D00078C6FF1F034B00EB8002134483F8351051
:10A1E000B2E600BF78C6FF1F034B00EB80021344AA
:10A1F00083F83610A8E600BF78C6FF1F034B00EBBC
:10A200008002134483F837109EE600BF78C6FF1F14
:10A21000034B00EB8002134483F8381094E600BF30
:10A2200078C6FF1F034B00EB8000184490F8340001
:10A23000704700BF78C6FF1F034B00EB8000184437
:10A2400090F83500704700BF78C6FF1F034B00EB46
:10A250008000184490F83600704700BF78C6FF1F92
:10A26000034B00EB8000184490F83700704700BFA4
:10A2700078C6FF1F034B00EB8000184490F83800AD
:10A28000704700BF78C6FF1F034B00EB400213442A
:10A2900083F82C101AE600BF78C6FF1F034B00EBB3
:10A2A0004002134483F82D1010E600BF78C6FF1F4C
:10A2B000034B00EB4002134483F82E1006E600BF68
:10A2C00078C6FF1F034B00EB4000184490F82C00A9
:10A2D000704700BF78C6FF1F034B00EB40001844D7
:10A2E00090F92D00704700BF78C6FF1F034B00EBAD
:10A2F0004000184490F82E00704700BF78C6FF1F3A
:10A30000034BC0EBC002134483F820109AE500BF52
:10A3100078C6FF1F034BC0EBC002134483F8211023
:10A3200090E500BF78C6FF1F034BC0EBC00213448B
:10A3300083F8221086E500BF78C6FF1F034BC0EBF1
:10A34000C002134483F823107CE500BF78C6FF1FCA
:10A35000034BC0EBC002134483F8241072E500BF26
:10A3600078C6FF1F034BC0EBC002134483F82510CF
:10A3700068E500BF78C6FF1F034BC0EBC002134463
:10A3800083F826105EE500BF78C6FF1F034BC0EBC5
:10A39000C000184490F82000704700BF78C6FF1F27
:10A3A000034BC0EBC000184490F82100704700BF79
:10A3B00078C6FF1F034BC0EBC000184490F8220082
:10A3C000704700BF78C6FF1F034BC0EBC0001844A6
:10A3D00090F82300704700BF78C6FF1F034BC0EB07
:10A3E000C000184490F82400704700BF78C6FF1FD3
:10A3F000034BC0EBC000184490F82500704700BF25
:10A4000078C6FF1F034BC0EBC000184490F826002D
:10A41000704700BF78C6FF1F9DF8000040EA422247
:10A42000064839B9C2601BB1C36843F48073C36086
:10A43000C06873E442F40032F4E700BF78C6FF1F3F
:10A440002DE9F84F334CDDF82890DDF82C801F46BD
:10A450002318054693F840308B469246C600042BDD
:10A4600031D8DFE803F0031A1F242900FFF77AFC34
:10A4700063190122751B254483F8402095F8263086
:10A48000012B32D022D3022B35D0B8F1000F02D0ED
:10A49000236888F80030BDE8F88FFFF7D3FC631914
:10A4A0000222E7E7FFF750FD63190322E2E7FFF717
:10A4B0000DFD63190422DDE7331A234493F8243099
:10A4C0000BB9FFF79BFC63190022D3E7BBF1000F28
:10A4D00003D023689B0C8BF80030BAF1000FD4D066
:10A4E00023689B0A8AF80030CFE7002FCDD023687D
:10A4F0009B0A3B60C9E71FB12368DB0B5B013B6034
:10A50000B9F1000FC1D02368C3F3842389F8003068
:10A51000BBE700BF78C6FF1F28B9034BDA7A12B930
:10A520000122DA721EE4704778C6FF1F20B9034B80
:10A53000D97A09B1D87215E4704700BF78C6FF1FF9
:10A54000062808D8DFE800F004080B0E11141700E5
:10A550000A4B1B680B607047084BDB69FAE7074B37
:10A560001B69F7E7054BDB6BF4E7044B1B6BF1E76B
:10A57000024B9B6AEEE7014BDB7AEBE778C6FF1FE5
:10A580000F4A1048002330B5194613705370141D3C
:10A590004FF0FF3544F82350C15401332F2BF9D12C
:10A5A000094B82F8C0101960084B82F8CC10196072
:10A5B000074BC2F8C410C2F8C810196030BD00BF04
:10A5C000BCC6FF1F7ACEFF1F5CD0FF1F78D0FF1FD5
:10A5D000E4CEFF1F13B5B94C63789A1F012A11D935
:10A5E0008C2B0FD0C02B0DD0C72B0BD003F16002EA
:10A5F000D2B2182A06D903F13402D2B2322A07D8CD
:10A60000D52B05D0A27832B10422AD4B1A7049E1A6
:10A61000A278022AF8D8A42B00F0698200F2A88060
:10A62000842B00F057814AD8062B00F07F8119D87F
:10A63000022B00F04F8107D8002B00F02A81012B5C
:10A6400000F032810322E0E7042B23D040F2628144
:10A65000D4F80310A078FFF706F9A278D4F8031015
:10A66000984B26E0802B00F014810ED80C2B00F0C4
:10A6700064810D2B00F08281072BE3D1A278924BED
:10A6800003EB4213E2789A720CE1822B00F08B818B
:10A6900040F20A81A178D4F80320490141F0060173
:10A6A00001F0E6010020FEF7AAFFA278D4F803101B
:10A6B000864B43F82210864B1344002227E1942B4B
:10A6C00000F03B8128D88A2B00F076810ED8862BAB
:10A6D000BED0C0F01F81872BB4D1A178D4F803205D
:10A6E000490141F00E0101F0EE011BE18D2B00F05C
:10A6F0007181932B00F042818C2BA3D1E178A0785B
:10A70000C1F10801C9B2FFF7B5FCA2786E4B03EBAB
:10A710004213E278DA72C5E0A02B00F0D3811BD897
:10A72000992B00F063819A2B00F07C81952B89D1C5
:10A73000A178490141F0140101AA01F0F4010020BF
:10A74000FEF7FDFFD4F803209DF80530002A00F045
:10A750004A8143F0040301E1A22B00F0C18140F2E1
:10A76000B881D4F80310A078C9B2FFF7C1FC99E012
:10A77000B52B00F017823ED8AC2B00F0E2811BD83D
:10A78000A82B00F0C9810BD8A62B00F0BE8140F2A7
:10A79000B581D4F80310A078C9B2FFF7D1FC81E0ED
:10A7A000AA2B00F0C78140F2BE81D4F80310A07834
:10A7B000C9B2FFF723FD75E0B02B00F0DE810BD8A6
:10A7C000AE2B00F0D38140F2CA81D4F80310A078F8
:10A7D000C9B2FFF795FD65E0B22B00F0DC81C0F057
:10A7E000D381B32B7FF42EAFD4F80310A078C9B275
:10A7F000FFF7B8FD56E0C72B00F0988022D8C02B99
:10A800003FF43CAF0ED8B72B00F0E581C0F0D48107
:10A81000B82B7FF417AFD4F80310A078C9B2FFF7B4
:10A820006FFC3FE0C22B00F01681C0F00D81C32BFE
:10A830007FF408AFA278244B03EB4213D4F8032033
:10A840005A602FE0D42B00F0268110D8D12B00F0D5
:10A850000981D22B00F00C81CC2B7FF4F3AEA278CF
:10A86000194B03EB4213D4F80320DA811AE0D62BFC
:10A8700000F02081C0F01781FE2B7FF4E3AE124B75
:10A88000A178D4F8032003EB411302B101221A731B
:10A8900008E0A178D4F80320490101F0E00100208C
:10A8A000FEF7BFFE02B010BDA178D4F80320490125
:10A8B00041F0020101F0E201F1E700BFDCCEFF1F31
:10A8C00070D0FF1F7CD0FF1FB8CDFF1F88D4FF1FA3
:10A8D000BCC6FF1FA178D4F80320490141F008014C
:10A8E00001F0E8010020FEF78AFEA178D4F80320E9
:10A8F0004901002A41F00601B8BF524201F0E601C9
:10A900000020FEF77CFEA278B74B1344012283F8A7
:10A91000CD20C7E7A178D4F80320490141F00A010E
:10A9200001F0EA010020FEF76AFEBBE7A278AF4B18
:10A9300003EB4213E2785A72B4E7A178490141F07F
:10A94000140101AA01F0F4010020FEF7F8FED4F88A
:10A9500003209DF8053072B143F002038DF80530F5
:10A96000A178490141F0140101AA01F0F40100208D
:10A97000FEF720FE96E723F00203EFE7A1784901F6
:10A9800041F0140101AA01F0F4010020FEF7D7FE06
:10A99000D4F803209DF8053012B143F00103DDE740
:10A9A00023F00103DAE7A178D4F80320490141F04C
:10A9B000040101F0E401B5E7A178490141F0140177
:10A9C00001AA01F0F4010020FEF7B9FEE3788DF84A
:10A9D0000630C5E7A178D4F80320490141F01A01F7
:10A9E00001F0FA019EE723F00403B7E7A1784901DB
:10A9F00041F0180101AA01F0F8010020FEF79FFEC6
:10AA00009DF80530E27823F00F0302F00F021343A4
:10AA1000A1788DF80530490141F0180101AA01F033
:10AA2000F801A4E7A178490141F0180101AA01F059
:10AA3000F8010020FEF783FE9DF80530E27803F070
:10AA40000F0343EA0213E3E7A278684B03EB4213D8
:10AA5000E2781A7226E7A378644AD4F803105B01FF
:10AA6000D1501FE7D4F80310A07805F0F9F919E7E1
:10AA7000A0785E4BE178D4F8032003EB401301F09B
:10AA80001F011A6105F0DCF9D4F80310A078491110
:10AA900005F0CEF906E7A278544B03EB4213D4F845
:10AAA00003205A61FEE6A278504B03EB4213E27892
:10AAB0009A77F7E6A2784D4B03EB4213D4F80320C4
:10AAC0009A83EFE6D4F80310A078C9B2FFF7DEFA54
:10AAD000E8E6D4F80310A078C9B2FFF7E1FAE1E69E
:10AAE000D4F80310A078C9B2FFF7FAFADAE6D4F87E
:10AAF0000310A078C9B2FFF70BFBD3E6D4F803101C
:10AB0000A078C9B2FFF70CFBCCE6D4F80310A0780C
:10AB1000C9B2FFF70DFBC5E6D4F80310A078C9B29F
:10AB2000FFF74EFBBEE6D4F80310A078C9B2FFF7DA
:10AB300051FBB7E6D4F80310A078C9B2FFF754FB75
:10AB4000B0E6D4F80310A078C9B2FFF761FBA27891
:10AB5000274B03EBC203D4F803205A71A2E6D4F8C2
:10AB60000310A078C9B2FFF78FFB9BE6D4F803105F
:10AB7000A07849B2FFF792FB94E6D4F80310A078CE
:10AB8000C9B2FFF7C7FB8DE6D4F80310A078C9B2AD
:10AB9000FFF7CAFB86E6D4F80310A078C9B2FFF726
:10ABA000CDFB7FE6A078114BD4F8032003EB4013D4
:10ABB0009A61FEF7DDF875E6A078D4F803200C4B17
:10ABC00043F83020002A7FF46DAE03EBC0035979BF
:10ABD000FFF71EFB66E6A278054B03EBC203D4F831
:10ABE00003201A715EE600BFBCC6FF1FB8CDFF1F71
:10ABF00024CDFF1F37B5C04DC04C6B789A1F012A7A
:10AC000011D98C2B0FD0C02B0DD0C72B0BD003F13B
:10AC10006002D2B2182A06D903F13402D2B2322A23
:10AC200007D8D52B05D0AA7832B10423237003B0FE
:10AC300030BDAA78022AF8D8A32B00F03F8200F298
:10AC4000BE80832B00F08B815BD8082B00F0A580A1
:10AC500021D8032B00F07C810ED8012B00F07181EC
:10AC600040F26681A978490141F0080101F0E8014C
:10AC70000020FEF77BFD62E1052B4ED0C0F06F8116
:10AC8000062B00F0FD80072B39D1AA789C4B03EBF3
:10AC900042139B7AF9E00C2B00F0668114D80A2B42
:10ACA00000F0788140F26F8101AA7C210020FEF73C
:10ACB00046FDAB785A00022393409DF806201342CC
:10ACC00014BF01230023E0E0802B00F0318110D875
:10ACD0000D2B14D1A978490141F0140101AA01F00A
:10ACE000F4010020FEF72BFD9DF8053003F0010371
:10ACF000CBE0812B00F02581822B00F056810323CD
:10AD00006AE1942B00F0308122D8872B00F0548127
:10AD100006D8852B00F01C81A4D9AA78794B20E1B4
:10AD20008C2B00F050810ED88A2BE8D1A9784901EC
:10AD300041F0140101AA01F0F4010020FEF7FFFC2C
:10AD40009DF80630A1E08D2B00F04881932BC0E7E1
:10AD50009C2B00F01F811AD8992B00F0468110D847
:10AD6000952BCCD1A978490141F0140101AA01F039
:10AD7000F4010020FEF7E3FC9DF80530C3F38003E7
:10AD800083E09A2B00F040819B2B8DD0B7E7A02B5E
:10AD900000F08C810AD89D2BB1D10020FEF7C9FCB0
:10ADA000AB785B00184100F00100C8E0A12B00F077
:10ADB0008181A22BA3D1A878FFF7CAF9BFE0B62BF7
:10ADC00000F0B98142D8AC2B00F094811AD8A72B9F
:10ADD00000F0808108D8A52B00F0788140F27281C4
:10ADE000A878FFF7DDF9AAE0A92B00F07B81C0F07D
:10ADF0007581AA2B00F07A81AB2B80D1A878FFF760
:10AE00002FFA9CE0B12B00F087810ED8AE2B00F01A
:10AE10007B81C0F07581AF2B00F07A81B02B7FF47D
:10AE20006EAFA878FFF7BCFA89E0B32B00F07C8105
:10AE3000C0F07681B42B00F07B81B52B7FF45FAF3F
:10AE4000AA782F4B03EB42139B691EE0CC2B00F03A
:10AE5000FD802CD8C12B00F0E58006D8B82B00F07F
:10AE60007581C0F06D81C02B0EE7C32B00F0E5802B
:10AE7000C0F0DE80C42B00F0E680C72B7FF43FAF2C
:10AE8000AA781F4B03EB42135B7A63601E4B1B785F
:10AE9000002B3FF4CCAE1D4B62681A601C4B002A9D
:10AEA00040F058811A6842F008021A60BFE6D22BBF
:10AEB00000F0EA8013D8CF2B00F0CE8005D8CE2B3F
:10AEC0007FF41DAFAA78134B4BE0D02B00F0D88055
:10AED000D12B7FF414AFA87804F0B6FF2FE0D52B68
:10AEE00000F0D88018D8D42B7FF409AFAA78044B8F
:10AEF00003EB42135B69C8E7DCCEFF1F70D0FF1F76
:10AF0000B8CDFF1F7CD0FF1F6BD0FF1F5CD0FF1F91
:10AF1000E4CEFF1F48CDFF1FD62B00F0C180FE2BD3
:10AF20007FF4EDAEAA788D4B03EB42131B7BACE7AD
:10AF3000A978490101F0E0010020FEF71FFE6060E2
:10AF4000A4E7A978490141F0020101F0E201F3E729
:10AF5000A978490141F00A0101F0EA0188E6AA78DE
:10AF60007F4B53F8223090E7A978490141F0140152
:10AF700001AA01F0F4010020FEF7E1FB9DF8053085
:10AF8000C3F3400381E70020FDF7D4FD003018BF74
:10AF90000120D4E701AA7C210020FEF7D0FBAA788B
:10AFA0009DF8063052001341A0E6A978490141F00E
:10AFB000040101F0E4015BE6A978490141F00E01CA
:10AFC00001F0EE0154E6AB782BB90020FFF770F8E2
:10AFD000C0F10800B3E70423237057E7A9784901BB
:10AFE00041F01A0101F0FA0142E6A978490141F065
:10AFF000180101AA01F0F8010020FEF7A0FB9DF85E
:10B00000053003F00F0340E7A978490141F018012A
:10B0100001AA01F0F8010020FEF791FB9DF8053030
:10B020001B0932E7AA784D4B03EB42131B7A2CE73E
:10B03000AB784A4A5B01D35827E7AA78474B03EB22
:10B0400042135B6821E7AA78464B8AE7AA78434B0C
:10B0500003EB4213DB8918E700236360424AAB78B5
:10B06000D15C09B1012161600021D1543F4AD15C1A
:10B0700019B1616841F0020161600021D15405E716
:10B08000AB783B4AD35C00E7AA78344B03EB42131E
:10B090001B69FAE6AA78314B03EB42139B7FF4E677
:10B0A000AA782E4B03EB42139B8BEEE6A878FFF7B2
:10B0B00007F844E7A878FFF70BF840E7A878FFF710
:10B0C0004FF83CE7A878FFF75BF838E7A878FFF778
:10B0D0005FF834E7A878FFF76BF830E7A878FFF758
:10B0E000A1F82CE7A878FFF7A7F828E7A878FFF7DA
:10B0F000ADF824E7AA781F4B03EBC2035B79C4E6E3
:10B10000A878FFF7DFF81AE7A878FFF7E5F816E761
:10B11000A878FFF73BF912E7A878FFF74BF90EE79D
:10B12000A878FFF751F90AE7A878FFF761F906E771
:10B13000AB78114AA6E7AA780E4B53F83230A4E652
:10B14000AA780C4B03EBC2031B799EE6A878FFF7A5
:10B150000FF8F4E61A6822F00802A6E6B8CDFF1F41
:10B1600088D4FF1F0CCDFF1FB0CDFF1F40CDFF1FA8
:10B17000B3CDFF1F24CDFF1F20CDFF1F38B58E4C50
:10B1800063789A1F012A0AD98C2B08D0C02B06D0CD
:10B19000C72B04D003F13402D2B2322A05D8A278E8
:10B1A00032B10422854B1A7038BDA278022AF8D831
:10B1B0009A2B29D8992B80F0C180822B00F0A48093
:10B1C00014D8062B00F0968005D8042B5FD0052BF1
:10B1D00074D00322E6E7072B22D00C3B012BF8D8D2
:10B1E0001421A078BDE83840FEF7CABB8C2B00F0D4
:10B1F0008D8003D8832B4AD0862BE9E78D2B00F076
:10B200009B80933B022BEAE7C72B73D01FD8C12B3F
:10B2100000F0A1800ED8B52B00F09280C02BD8D1C1
:10B22000A47860014A30FEF768F8654B03EB4413DD
:10B23000987238BDC22B00F09880C32BC9D1A0787A
:10B240006049023040010422014410447FE0D42BC5
:10B2500000F09A800CD8CC2B00F08E80D22BB8D185
:10B26000A0785949023040010144042210306EE0B8
:10B27000D62B00F09980C0F08F80FE2BA9D1A0784A
:10B28000524902304001014401220C305FE00621A6
:10B29000A078FEF775FBA578690141F0060101F081
:10B2A000E6010020FEF762FA494BA27843F8250038
:10B2B000484B1344002283F8CD2038BDA0780C21E0
:10B2C000FEF75EFBA578690141F00C0101F0EC018D
:10B2D0000020FEF74BFA404A3E4B42F82500A0788A
:10B2E0000344002183F8CD10BDE8384052F8201007
:10B2F000FEF7B9BAA47860014930FDF7FEFF304B84
:10B3000003EB4413587238BD04216AE7A378002B7D
:10B310007FF447AF2A4D4B2005F10B010122FEF7C8
:10B3200005F8A07805EB4015E97AC1F10801C9B22A
:10B33000BDE83840FEF79EBE1A2152E7182150E7BB
:10B34000A078264902304001014404221830BDE8AB
:10B350003840FDF7EBBFA47860014830FDF7CDFF22
:10B36000174B03EB4413187238BDA0781C49023008
:10B37000400104220144EAE7A0781A490230400162
:10B38000014402220E30E2E7A07817490230400162
:10B39000014404221430DAE7A07814490230400155
:10B3A000014401221E30D2E7A07811490230400149
:10B3B000014402221C30CAE7DCCEFF1F70D0FF1F01
:10B3C000B8CDFF1F7CCDFF1F88CDFF1F84CDFF1F91
:10B3D00088D4FF1FBCC6FF1F7CD0FF1F90CDFF1F6E
:10B3E00078CDFF1F86CDFF1F8CCDFF1F96CDFF1F91
:10B3F00094CDFF1F38B5994A9378022B144600F07C
:10B400002681032B00F03881002B40F00E82537808
:10B410004E2B00F0C18031D8462B00F08F8012D81F
:10B42000422B7BD006D8402B6CD0412B71D003220D
:10B430008B4B65E0442B76D0452BF8D1894BD178E6
:10B440005971052061E04B2B00F096800CD8472BFA
:10B450007CD0492BEBD1D278824B002A40F08780F8
:10B46000DA75D97D172050E04C2B00F090804D2BE1
:10B47000DDD17C4BD1785975152046E0542B00F076
:10B48000BD801BD8512B00F0A48009D84F2B00F0B1
:10B490008E80502BCBD1734BD1789975162034E028
:10B4A000522B00F0A380532BC1D16E4DD2F8033044
:10B4B0002946042241F8103F10204FE0832B00F072
:10B4C000B58014D8552B00F0A580562BAFD1D2F8FB
:10B4D00003300F2B00F2A981D1780020FEF7A2F9EA
:10B4E0006049E37801F8243F0122242022E0852BE3
:10B4F00000F0A780C0F0A080FF2B98D1D2785A4BE3
:10B500001A7038BDD17840F2FF70BDE83840FDF7C1
:10B510001BBE544BD17819700020F6E7514BD178FF
:10B5200059700120F1E74F49D2F8033041F81C3F30
:10B5300004221C20BDE83840FDF765BE4949D2F819
:10B54000033041F80C3F04220C20F3E7454DD2F8BC
:10B5500003302946042241F8083F0820FDF753FE36
:10B560002A8A29896879BDE8384004F0B1BA3C4993
:10B570000122DA754A6074E73A4CD178E170032011
:10B58000FDF7E2FDE078BDE83840FDF733B9354B13
:10B59000D17899700220B8E7324CD2F80300E084E9
:10B5A000FDF742FB022204F126012620C2E7D2F871
:10B5B00003102C4CC9B219206176FDF7C5FD617EE0
:10B5C00011F0010118BF01210020BDE83840FEF74D
:10B5D00011BB244D2A7DD20704D5E378DB0701D4C3
:10B5E000FDF719FDE178297514208EE71D49D2F881
:10B5F000033041F8203F042220209BE7D2F803309B
:10B60000012B00F212811749D37801F81A3F012269
:10B610001A208FE7D2F80330012B00F2068111497E
:10B62000D37801F81B3F01221B2083E70F4BD2F890
:10B630000320C3F8D02038BD0D4BD2F803201A6088
:10B6400038BD0A4BD2F80320C3F8D42038BD517856
:10B65000084BD2F8032043F8212038BDDCCEFF1F71
:10B6600070D0FF1F0CC0FF1F6AD0FF1FBCC6FF1F9A
:10B670006CD0FF1F88D0FF1F53782E2B3FF6D7AE1C
:10B6800001A252F823F000BF45B7000059B70000EF
:10B690006DB700002FB400002FB400002FB40000DD
:10B6A0002FB400002FB400002FB4000081B70000B9
:10B6B0008BB7000095B700002FB400002FB4000036
:10B6C0002FB400002FB400002FB400002FB40000EE
:10B6D0002FB400002FB400002FB400002FB40000DE
:10B6E0002FB400002FB400002FB400002FB40000CE
:10B6F0002FB400009FB70000ADB70000BBB700003B
:10B70000C3B70000CBB70000D3B700002FB40000D0
:10B710002FB400002FB400002FB400002FB400009D
:10B720002FB40000DBB70000E5B70000EFB7000062
:10B73000F9B7000003B800000DB8000017B800000A
:10B7400021B800003A4BD4F803201A60FCF7DCFF64
:10B75000384BC3F8D80038BD354BD4F803205A60B5
:10B76000FCF7D2FF334BC3F8DC0038BD304BD4F8C4
:10B7700003209A60FCF7C8FF2E4BC3F8E00038BDE9
:10B780002B4BD4F80320DA6038BD294BD4F80320C2
:10B790001A6138BD264BD4F803205A6138BDD4F85D
:10B7A00003100020BDE83840FEF747B9D4F8031075
:10B7B0000020BDE83840FEF76AB9D4F80310012034
:10B7C000F0E7D4F803100120F3E7D4F803100220C7
:10B7D000E8E7D4F803100220EBE7154BD4F8032078
:10B7E0009A6138BD124BD4F80320DA6138BD104B92
:10B7F000D4F803201A6238BD0D4BD4F803205A62E6
:10B8000038BD0B4BD4F803209A6238BD084BD4F8EE
:10B810000320DA6238BD064BD4F803201A6338BD22
:10B82000034BD4F803205A6338BD042200E600BF5E
:10B8300028CEFF1FBCC6FF1F2DE9F047214EB3786D
:10B84000022B3AD8DFF88880DFF88890DFF888A0EC
:10B850000025B278ECB2A24209D01B4B03EB421296
:10B86000927F2AB303EB45139B7F934220D100279D
:10B8700001232146640105F808300222384664B2EB
:10B8800005F8097005F80A70FDF786FF44F0060117
:10B8900040F2FF7201F0E601384644F00804FDF77B
:10B8A000AEFED6F8032004F0E8013846FDF7A7FE07
:10B8B0000135032DCDD1BDE8F087044B04221A7069
:10B8C000BDE8F087DCCEFF1FB8CDFF1F70D0FF1F93
:10B8D00089C7FF1FB0CDFF1F40CDFF1F2DE9F047E7
:10B8E000224EB378022B3BD8DFF88C80DFF88C90A7
:10B8F000DFF88CA00025B278ECB2A24209D01C4B34
:10B9000003EB4212927F32B303EB45139B7F9342CA
:10B9100021D1002701232146640105F808300222C5
:10B92000384664B205F8097005F80A70FDF734FF6F
:10B9300044F0060140F2FF7201F0E6013846FDF7DF
:10B940005EFED6F8032044F00804524204F0E801F9
:10B950003846FDF754FE0135032DCCD1BDE8F08704
:10B96000044B04221A70BDE8F08700BFDCCEFF1F35
:10B97000B8CDFF1F70D0FF1F89C7FF1FB0CDFF1FBD
:10B9800040CDFF1F2DE9F041164E174FDFF86080C4
:10B990000025B278ECB2A24209D0144B03EB42125C
:10B9A000927FCAB103EB45139B7F934214D120468B
:10B9B00003F0BCFF022221460020FDF7EDFE6101ED
:10B9C00041F0080101F0E8010020FDF79BFE012392
:10B9D000EB55002305F808300135032DD9D1BDE81A
:10B9E000F08100BFDCCEFF1F89C7FF1FB8CDFF1F4E
:10B9F00040CDFF1F2DE9F047804616460F4600292F
:10BA00004DD000284BD0814249D0540164B244F05B
:10BA10000605EDB229460020FEF7B0F844F00C010F
:10BA200001F0EC0182460020FEF7A8F8814640466E
:10BA300006F034FF0446384606F030FF0146204643
:10BA400007F038F80746504606F028FF394607F059
:10BA500031F807F041F90446484606F01FFF394621
:10BA600007F028F807F038F9002C08BF01240D4929
:10BA7000002814BF80464FF00108384607F004F94B
:10BA800018B141463046FDF7EEFE22462946002019
:10BA9000FDF7C7FD044A3244012382F8CD30BDE8EA
:10BAA000F08700BF0000A041BCC6FF1F70B50E4C60
:10BAB0000444054694F8CD30A3B1C6B20B4B7101D6
:10BAC00041F0060153F8202001F0E6010020FDF7C7
:10BAD00096FD074B304653F82510FDF7C4FE0023B2
:10BAE00084F8CD3070BD00BFBCC6FF1F88D4FF1FD7
:10BAF0007CD0FF1F2DE9F04FC94CA078022885B0FB
:10BB000003D96378022B40F0B0806378032B00F2F6
:10BB1000C381DFE813F004003C007D009301DFF8EF
:10BB20000C83DFF81493BF4F0025A278AA4209D0F6
:10BB3000BD4B03EB4212927F1AB303EB45139B7F7D
:10BB400093421ED12846FFF7B1FF012303FA05F205
:10BB50005FFA85FA3B7800264FEA4A1123EA02038E
:10BB600001F0E001D4F8032005F80860304605F83C
:10BB700009603B70FDF755FD324651463046FDF7F2
:10BB80000BFE0135032DD0D105B0BDE8F08FDFF8F5
:10BB9000A8B2DFF890920025A278AA4209D0A24B61
:10BBA00003EB4212927F7AB303EB45139B7F9342E0
:10BBB0002AD128465FFA85FAFFF778FF4FEA4A183C
:10BBC0009A4B00265FFA88F8EE5448F0020105F817
:10BBD0000B603046FDF7D2FF012202FA05F1D4F8DE
:10BBE000037099F80020074422EA010289F8002036
:10BBF00041463A463046FDF714FD3246514630463E
:10BC0000FDF7CAFD8A4B5F600135032DC4D1BBE748
:10BC1000D4F803301E2B28DC10F0C00529D10228EF
:10BC200023D803EB43030344824A7E4E52F8237029
:10BC3000FFF73CFFA1787D4B5D547F4B5D540123A2
:10BC400003FA01F0337823EA0003337049013A46DE
:10BC5000284601F0E001FDF7E4FCA1782A462846D9
:10BC600005B0BDE8F04FFDF797BD0422704B1A7088
:10BC70008AE7402D40F09D800025019502950395AF
:10BC80002A4640FA02F1C90706D504A9294401351C
:10BC9000032D01F8102C02D00132032AF1D1DFF874
:10BCA0009491002703EB4306AF423DD1012F0BDDFA
:10BCB000022F019E029D56D1AE424FDD9DF801201C
:10BCC00029463046FFF796FE5A4FDFF86081DFF8CD
:10BCD00068910025A3782B41DA0721D5D4F80330E9
:10BCE000504803EB43032B445FFA85FA57F82320AF
:10BCF000012303FA05F10378002623EA01034FEA42
:10BD00004A11037001F0E001304605F8086005F8BB
:10BD10000960FDF786FC324651463046FDF73CFD92
:10BD20000135032DD6D12FE71DF807804046FFF7D8
:10BD3000BDFE4FEA481141F0020101F0E20100208E
:10BD4000B044FDF71BFF59F82830C01A002801AB9A
:10BD5000B8BF404243F827000137A5E79DF800200F
:10BD600031462846AEE7AE42039F16DDBE4209DDEE
:10BD70009DF8012029463046FFF73CFE9DF8022041
:10BD800039469EE79DF8002031463846FFF732FEDF
:10BD90009DF801202946384694E7BD4231469DF87A
:10BDA0000020F2DD2846FFF725FE9DF802203946E7
:10BDB000D7E7802D7FF459AFDFF878901B4FDFF87D
:10BDC00078800025A3782B41DB0724D5D4F80330F5
:10BDD00003EB43032B44284659F823A0FFF766FEE4
:10BDE000104A012303FA05F113785FFA85FB002658
:10BDF00023EA01034FEA4B11137001F0E0015246B0
:10BE00003046EE5505F80860FDF70BFC3246594602
:10BE10003046FDF7C1FC0135032DD3D1B4E600BF98
:10BE2000DCCEFF1F19CDFF1FB8CDFF1F40CDFF1F78
:10BE300070D0FF1FE8CEFF1FB0CDFF1F02283FF6D6
:10BE400014AFD4F803301E2B3FF70FAF400140F082
:10BE5000020101F0E2010020FDF790FED4F803306A
:10BE6000A1780E4A03EB43030B44002552F82360EC
:10BE700006440846FFF71AFEA178094B09485D54AD
:10BE8000094B5D54012303FA01F2037823EA02030C
:10BE9000037049013246DBE60322E7E6E8CEFF1FE6
:10BEA00040CDFF1F19CDFF1FB0CDFF1F2DE9F3417E
:10BEB000C24EC3493378D6F803004B706422292B55
:10BEC0000A70486034460D4601F07F8100F2E6803A
:10BED000142B00F0398559D80A2B00F0D08222D8D3
:10BEE000052B00F0D08111D8022B00F0C38105D8BA
:10BEF000012B00F0BA8102232B70B8E1032B00F074
:10BF0000BC81042BF7D1FFF7F5FDB0E1072B00F062
:10BF1000C081C0F0BB81082B00F0AE82092BEAD1B2
:10BF2000FFF768FAA3E10F2B00F0AC8413D80C2BB9
:10BF300000F03A84C0F023840D2B00F047840E2BD0
:10BF4000D9D1B378002B00F08084022B00F08484D8
:10BF500004230B708BE1112B01F04184C1F0388474
:10BF6000122B01F04384132BC5D17278954B092A0B
:10BF700000F2DD84DFE812F0BB04BF04C204C50494
:10BF8000C904CF04D204D504D804BD041F2B00F08B
:10BF9000FF864DD8192B00F09B8519D8162B00F081
:10BFA0007F85C0F0F084172B00F07F85182BA2D17D
:10BFB000854AD2F8C830002B00F05981013BC2F805
:10BFC000C83002EB8303D3F8E430C2F8C4304EE14A
:10BFD0001B2B00F09D85C0F08B851C2B00F09C86F0
:10BFE0001E2B88D173781E2B00F2D883B678022ED0
:10BFF00000F2988603EB43023244744C44F822006A
:10C00000734A927E002A00F03281002B00F02F81CB
:10C01000032111FB03610C20013B434303F5C36083
:10C02000042204EB810102FB0600FDF7ECF81EE19F
:10C03000242B00F0B58711D8212B00F05387C0F0D6
:10C04000F586222B00F0A487232B7FF454AF5D4BA1
:10C050001B68C6F80330FFF7CDF908E1262B00F086
:10C06000EB87C0F0D087272B01F00E80282B7FF4C0
:10C0700042AFFF2800F3FB8073780B2B01F2A18005
:10C08000DFE813F014081F082A08350841084F0894
:10C090005A0865087008790881088D08432B01F05B
:10C0A000E08469D8332B01F0728332D82E2B01F053
:10C0B00040831CD82B2B01F0AD81C1F015812C2BB6
:10C0C00001F036822D2B7FF416AF73780B2B01F223
:10C0D0002C83DFE813F0C90AD20ADB0AE40AEE0A6D
:10C0E000FA0A030B0C0B150B1E0B2A0B240B302B1F
:10C0F00001F03283C1F02583312B01F03983322BDB
:10C100007FF4F9AE2F4B1B68C6F80330FFF7E6FB50
:10C11000ADE0382B01F0758313D8352B01F048833F
:10C12000C1F03B83362B01F04E83372B7FF4E3AE17
:10C13000284B1B68FF2B00F29A80274A42F8230005
:10C1400095E0402B01F085840DD8392B7FF4D3AED8
:10C15000204B1B68FF2B00F28A801A4A11681E4A86
:10C1600042F8231083E0412B01F07784422B7FF4C7
:10C17000C2AE02F059FB7AE0842B01F0A28436D8DB
:10C18000502B01F057830DD8452B01F07284C1F07C
:10C190006C84462B01F07184472B7FF4ACAE02F027
:10C1A00048FB64E0812B01F06C8417D8802B7FF46E
:10C1B000A2AE054B002283F8C02058E0DCCEFF1F62
:10C1C00070D0FF1F5CD0FF1FBCC6FF1FE8CEFF1F53
:10C1D0000CC0FF1F78D0FF1F88D0FF1F822B01F0FB
:10C1E0006A84832B7FF487AEFEF7CAF93FE0892B80
:10C1F00001F0288516D8862B01F07E84C1F0768464
:10C20000872B01F0E384882B7FF475AE7378012BC4
:10C2100001F0C184C1F0AC84022B01F0C58403237A
:10C220000B7024E08D2B01F05E850FD88A2B01F076
:10C2300022858C2B7FF45FAE7678002E01F034855A
:10C24000012E01F0418503230B7010E0F22B01F069
:10C250009985FF2B7FF44FAE40F2D243984206D12E
:10C26000AD4B012283F8602101E0FFF7E5FA02B04F
:10C27000BDE8F081FFF732FBF9E7B378022B19D85C
:10C28000FFF780FBF3E7FEF7A5F9F0E7FEF7B2FC56
:10C29000EDE773789A1F012A0AD98C2B08D0C02B9E
:10C2A00006D0C72B04D003F13402D2B2322A04D80C
:10C2B000A2782AB104232B70D9E7B278022AF9D8E0
:10C2C0009A2B25D8992B80F08D80822B76D013D88D
:10C2D000062B69D006D8042B5CD0052B5FD0032336
:10C2E0002B70C4E7072B1DD00C3B012BF7D8142172
:10C2F000A078FDF769FBBAE78C2B64D003D8832BB9
:10C3000048D0862BEAE78D2B67D0933B022BEDE7D5
:10C31000C72B49D01ED8C12B73D00DD8B52B66D0F2
:10C32000C02BDCD1A0787D4B03EB40134001997A00
:10C330004A30FCF709FF9AE7C22B6CD0C32BCED151
:10C34000A078774902304001042201441044FCF7F0
:10C350005AFF8CE7D42B71D00DD8CC2B64D0D22BC4
:10C36000BDD1A0786F490230400101440422103051
:10C37000FCF749FF7BE7D62B74D069D3FE2BAED1F7
:10C38000A078694902304001014401220C30FCF7D9
:10C390003AFF6CE70621A078FDF716FB67E70C2152
:10C3A000A078FDF711FB62E7A0785C4B03EB40132C
:10C3B0004001597A4930FCF7C7FE58E70421A078BC
:10C3C000FDF702FB53E7A378002B7FF473AF012244
:10C3D00056494B20FCF717FF49E71A21A078FDF7D3
:10C3E000F3FA44E71821A078FDF7EEFA3FE7A078CA
:10C3F0004F4902304001014404221830FCF703FF8A
:10C4000035E7A078454B03EB40134001197A4830DB
:10C41000FCF79AFE2BE7A07846490230400104223F
:10C420000144FCF7F0FE22E7A078434902304001C6
:10C43000014402220E30FCF7E6FE18E7A0783F49DF
:10C4400002304001014404221430FCF7DCFE0EE708
:10C45000A0783B4902304001014401221E30FCF724
:10C46000D2FE04E7A078374902304001014402229D
:10C470001C30FCF7C8FEFAE6FEF780FEF7E6B3785C
:10C48000022B00F0D780032B00F0D980002B40F066
:10C490006F817378502B00F09F8025D8472B00F0D8
:10C4A0008B8011D8422B7ED006D8402B61D0412BF7
:10C4B00075D003232B7061E0452B77D079D8442BBE
:10C4C000F7D1214BDB696CE04C2B7ED006D8492B91
:10C4D00075D04B2BEDD11C4BDB7862E04E2B1A4B09
:10C4E00078D075D95B7E5CE0802B00F084802DD8FD
:10C4F000532B77D006D8512B71D0522BD9D1124B58
:10C500001B6A4EE0552B73D06FD3562BD1D10E4BF7
:10C5100093F8243045E000BFBCC6FF1FB8CDFF1F15
:10C520007CCDFF1F88CDFF1F84CDFF1FC3CDFF1F14
:10C5300090CDFF1F78CDFF1F86CDFF1F8CCDFF1F35
:10C5400096CDFF1F94CDFF1F0CC0FF1F832B5DD026
:10C5500007D8812B53D0822BABD1A64BD3F8C43054
:10C560001FE0852B59D055D3FF2BA2D1A24B1B78AE
:10C5700027E040F2FF70FCF7C0FE68609F4B1B781D
:10C58000002B3FF474AE9E4B6A681A609D4B002AE4
:10C5900040F0F0801A6842F008021A6067E69A4B91
:10C5A0001B786B60EAE7984B5B78FAE7964B5B7910
:10C5B000F7E7954BDB68F4E7934B9B68F1E7924B09
:10C5C000DB7D003318BF0123EBE78F4B9B78E8E757
:10C5D0005B7DE6E7DB8CE4E78B4B9B7DE1E78A4BF9
:10C5E0001B7DDEE7884B1B69DBE7874B9B7ED8E72B
:10C5F000854BDB7ED5E77F4B93F8C030D1E77D4B91
:10C6000093F8C0301A1F53425341CAE7794BD3F80D
:10C61000D030C6E77D4B1B68C3E7764A7C48D2F82A
:10C62000D43043F2390100FB0313C2F8D43023F0B5
:10C630000043B6E77278774B53F82230B1E773784E
:10C640002E2B3FF636AF01A252F823F009C70000A7
:10C650000DC7000013C70000B3C40000B3C400003E
:10C66000B3C40000B3C40000B3C40000B3C40000EE
:10C6700017C700001BC700001FC70000B3C400009D
:10C68000B3C40000B3C40000B3C40000B3C40000CE
:10C69000B3C40000B3C40000B3C40000B3C40000BE
:10C6A000B3C40000B3C40000B3C40000B3C40000AE
:10C6B000B3C40000B3C4000025C700002DC70000AC
:10C6C00035C7000039C700003DC7000041C7000062
:10C6D000B3C40000B3C40000B3C40000B3C400007E
:10C6E000B3C40000B3C4000045C700004BC700003E
:10C6F0004FC7000053C7000059C700005FC70000C4
:10C7000065C700006BC70000434B84E7424B5B6882
:10C7100047E7414B51E7404B4CE73F4B63E73E4B0C
:10C720005B693EE70020FDF7DCF926E70020FDF716
:10C73000EDF922E70120F6E70120F8E70220F2E711
:10C740000220F4E7344B9B692BE7334BBAE6324BBC
:10C75000D6E6314B5B6A24E72F4B9B6A21E72E4BD1
:10C76000DB6A1EE72C4B1B6B1BE72B4B5B6B18E745
:10C7700004239FE61A6822F008021A6077E5B3786E
:10C78000022B0ED17078372808D800F5A7702349FE
:10C79000800004220144FCF736FD68E503232B707A
:10C7A00065E504230B7062E5B378022B0BD170783A
:10C7B0003728F3D800F5A7701849800004220144F7
:10C7C000FCF7B4FD53E504230B7050E5B078022864
:10C7D0003FF670AD7378012B08D004D3022B1FD025
:10C7E00003230B7043E503F099F840E503F09EF84E
:10C7F0003DE500BFBCC6FF1F6AD0FF1F6BD0FF1F07
:10C800005CD0FF1FE4CEFF1F0CC0FF1F6CD0FF1FCA
:10C810006D4EC64188D0FF1F28CEFF1F50CBFF1F93
:10C8200003F08CF89A4B68601B78002B3FF41FAD27
:10C83000984B1860984B1A6818B942F008021A60B1
:10C8400015E522F008021A6011E57378002B7FF4D9
:10C850000EADFCF753FA0AE573781F2B08D818B908
:10C860001846FCF731F902E51846FCF709F9FEE431
:10C87000FF2B7FF4FCAC431C04BF864B1868FCF70D
:10C8800047F9F4E4B378012B24D004D3022B25D04C
:10C8900004230B700AE07078092803D8FCF74AF9E2
:10C8A000686003E00A2810D100234B60784B1B78A6
:10C8B000002B3FF4DCAC774B6A681A60764B8AB980
:10C8C0001A6842F008021A60D1E4FF28EED1FCF7A2
:10C8D0009BF9E5E7707803F0C9F8E1E77078FCF7B9
:10C8E0005DF9DDE71A6822F008021A60BFE41A68F1
:10C8F000104418601BE01A68101AFAE71A685043CF
:10C90000F7E71A6892FBF0F0F3E7196891FBF0F291
:10C9100000FB1210EDE71A681040EAE71A681043AE
:10C92000E7E71A685040E4E71A68D2431A601A68C9
:10C93000594B22B91A6842F008021A6097E41A6843
:10C9400022F008021A6092E4524B534A19681368A5
:10C9500088420ADA23F0030343F0040313601368E8
:10C9600069B943F00803136081E40BBF23F00603A9
:10C9700023F0050343F0010343F00203EEE723F045
:10C980000803136073E473780C2B3FF670ACDFE898
:10C9900003F0071019222B343E475059626B750083
:10C9A0003D4B1B681F077FF562AC3C4BC3F8C400CE
:10C9B0005DE4394B1B681E073FF559AC374BC3F894
:10C9C000C40054E4344B1B68DD077FF550AC334B97
:10C9D000C3F8C4004BE4304B1B68DC073FF547ACA1
:10C9E0002E4BC3F8C40042E42B4B1B6859077FF55C
:10C9F0003EAC2A4BC3F8C40039E4274B1B6813F044
:10CA0000050F3FF434AC254BC3F8C4002FE4224B90
:10CA10001B689A077FF52BAC204BC3F8C40026E4B3
:10CA20001D4B1B689B073FF422AC1C4BC3F8C40092
:10CA30001DE4194B1B68DF067FF519AC174BC3F8D3
:10CA4000C40014E4144B1B689E067FF510AC134B16
:10CA5000C3F8C4000BE4104B1B685D067FF507AC00
:10CA60000E4BC3F8C40002E40B4B1B681C067FF599
:10CA7000FEAB0A4BC3F8C400FFF7F9BB064B1B68BB
:10CA8000D9057FF5F4AB054BC3F8C400FFF7EFBB46
:10CA90006BD0FF1F5CD0FF1FE4CEFF1FBCC6FF1F83
:10CAA000B64BC3F8C400FFF7E2BBB44BD3F8C820C1
:10CAB000072A3FF6DCAB511C03EB8202C3F8C81017
:10CAC000D3F8C410C2F8E410C3F8C400FFF7CFBB1A
:10CAD00073782E2B04D8AA4A0121D154FFF7C7BB83
:10CAE000FF2B7FF45BAEA54B01221A70FFF7BFBB93
:10CAF00073782E2B04D8A24A0021D154FFF7B7BB7C
:10CB0000FF2B7FF44BAE9D4B00221A70FFF7AFBB9B
:10CB10009A4D95F8CC309BB9421C04BF994A1068D5
:10CB20004FF00A030BBF43435843C5F80431C5F81F
:10CB30000401FBF7E9FD0123C5F8080185F8CC30B5
:10CB40006378042B3FF693ABDFE803F003487AB039
:10CB50001B00FBF7D9FDD5F80831C01A0028D5F81D
:10CB60000431B8BF4042984295BFD5F8C430002385
:10CB700003F1FF3385F8CC3098BFC5F8C430FFF718
:10CB800076BBA07802F0DAFE40B97F4A85F8CC0087
:10CB9000136823F010031360FFF769BBD5F8043165
:10CBA000ABB1FBF7B1FDD5F80831C01A0028D5F8B4
:10CBB0000431B8BF4042984209D9734A002385F82E
:10CBC000CC30136843F010031360FFF750BBD5F867
:10CBD000C430013BC5F8C430FFF749BB0020FCF767
:10CBE000A8FDA3785B00184110F0010409D0664A43
:10CBF000002385F8CC30136823F010031360FFF78F
:10CC000036BBD5F80431A3B1FBF77EFDD5F808316A
:10CC1000C01A0028D5F80431B8BF4042984208D95C
:10CC2000594A85F8CC40136843F010031360FFF7AE
:10CC30001EBBD5F8C430013BC5F8C430FFF717BBA5
:10CC40006A467C210020FCF77AFDA3789DF802401B
:10CC50005A00022393401C4009D04B4A002385F818
:10CC6000CC30136823F010031360FFF700BBD5F836
:10CC70000431A3B1FBF748FDD5F80831C01A0028EC
:10CC8000D5F80431B8BF4042984208D93E4A85F8E9
:10CC9000CC40136843F010031360FFF7E8BAD5F8EF
:10CCA000C430013BC5F8C430FFF7E1BA6A467C21C5
:10CCB0000020FCF744FDA2789DF802305200134199
:10CCC00013F0010409D0304A002385F8CC301368F2
:10CCD00023F010031360FFF7CABAD5F80431A3B1EB
:10CCE000FBF712FDD5F80831C01A0028D5F8043139
:10CCF000B8BF4042984208D9234A85F8CC4013680F
:10CD000043F010031360FFF7B2BAD5F8C430013B0B
:10CD1000C5F8C430FFF7ABBA184B002283F8C02027
:10CD2000FFF7A5BAFF2E7FF4C5AA184E73B90C25DC
:10CD3000002405F20C6729193819042231440434FF
:10CD4000FCF761FA0C2CF6D10C35F1E700254FF019
:10CD500003080C27607818FB00510138784300F570
:10CD6000C36000EB8500042206EB81010135FCF76E
:10CD70004AFA032DEED1FFF77ABA00BFBCC6FF1FF7
:10CD80007ACEFF1F5CD0FF1FE4CEFF1FE8CEFF1F4F
:10CD900073781E2B3FF602ADB278022A1BD803EB44
:10CDA000430313449D4A52F823209D4B4A601B784D
:10CDB000002B3FF45CAA9B4B1A609B4B2AB91A6864
:10CDC00042F008021A60FFF752BA1A6822F008020D
:10CDD0001A60FFF74CBAFF2A7FF46CAA8F4E73B922
:10CDE0000C25002405F20C67291938190422314456
:10CDF0000434FCF79BFA0C2CF6D10C35F1E7002536
:10CE00004FF003080C27607818FB00510138784375
:10CE100000F5C36000EB8500042206EB81010135BB
:10CE2000FCF784FA032DEED1FFF721BA76781E2E97
:10CE30003FF6B4ACA7783B0630D5784FDFF8F481E5
:10CE40000025A3782B41DE070DD56901667841F0F6
:10CE5000020101F0E2010020FCF790FE06EB46061D
:10CE60002E4447F8260098F81A3093B16278531E82
:10CE7000D9B227290DD80C200321584311FB0251A8
:10CE800000F5C360042207EB810100EB8500FCF78D
:10CE9000BAF90135032DD4D1FFF7E9B9022F3FF6D6
:10CEA00009AA790141F0020101F0E2010020FCF73A
:10CEB00065FE06EB4606594D63783E44032145F86E
:10CEC0002600A0785A1E11FB03010C23534303F5DF
:10CED000C363042205EB810102FB0030FCF793F9E8
:10CEE000FFF7C5B972784F4B0A2A0CD8DFE802F079
:10CEF00006151A1F252D32373C4145004B491A684B
:10CF000009680A441A601A68474B002A3AD11A681D
:10CF100042F008021A60FFF7AAB944491A68096882
:10CF2000521AEFE7414A196812684A43EAE73F4953
:10CF30001A68096892FBF1F2E4E73C4A1868116844
:10CF400090FBF1F201FB1202DCE738491A6809682C
:10CF50000A40D7E735491A6809680A43D2E73349D6
:10CF60001A6809684A40CDE730490A68D2430A6026
:10CF7000C9E719682D4A1160C5E72C4A196810687D
:10CF80001860F8E71A6822F008021A60FFF76FB914
:10CF9000244B1B68C6F80330FDF71CFBFFF767B98D
:10CFA0007378052B3FF663A9DFE803F0030A111835
:10CFB0001F261D4A136803F00F031360FFF757B9CC
:10CFC000194A136823F010031360FFF750B9164A8B
:10CFD000136823F020031360FFF749B9124A13685E
:10CFE00023F040031360FFF742B90F4A136823F0A0
:10CFF00080031360FFF73BB90B4A136823F4807377
:10D000001360FFF734B972782E2A3FF6C7AB084B8E
:10D0100003EB82035860FFF72AB900BFE8CEFF1F79
:10D020006BD0FF1F5CD0FF1FE4CEFF1F78D0FF1F27
:10D03000BCC6FF1F0CC0FF1FB24BB34AD3F80C1184
:10D040001160B24AD3F810111160D3F81421C3F85B
:10D05000C420AF4AD3F818111160D3F81C2183F80B
:10D06000CC20D3F82021C3F80821D3F82421C3F819
:10D07000042193F82811A74A505C08B101205054AC
:10D0800000225A70FFF7F3B8B278022A3FF612A9CD
:10D0900073781E2B3FF682AB03EB430313449A4A8B
:10D0A00011689D4A42F82310FFF7E1B89B4BB17815
:10D0B00053F8200053F82120024443F82120FFF7C1
:10D0C000D6B8964BB17853F8200053F82120121AA5
:10D0D00043F82120FFF7CBB8904BB17853F82020CC
:10D0E00053F82140624343F82120FFF7C0B88B4B2F
:10D0F000B17853F8200053F8212092FBF0F243F866
:10D100002120FFF7B4B8854BB17853F8200053F8CD
:10D11000214094FBF0F200FB124243F82120FFF77C
:10D12000A6B87E4BB17853F8200053F82120024076
:10D1300043F82120FFF79BB8784BB17853F82000D3
:10D1400053F82120024343F82120FFF790B8734B96
:10D15000B17853F8200053F82120424043F82120B1
:10D16000FFF785B86D4AB17852F82030DB4342F8BA
:10D170002130FFF77CB8694BB27853F8201043F8A0
:10D180002210FFF774B8654BB27853F8204053F87B
:10D19000221043F8224043F82010FFF768B85F4B95
:10D1A000B27853F8222053F820309A4240F34A8252
:10D1B000574A136823F0030343F004031360FFF797
:10D1C00056B803230B70FFF752B873780B2B00F29D
:10D1D0008780DFE803F006111C2733414C57626B50
:10D1E000737EB1784D4A484852F8213000680344B4
:10D1F00042F82130FFF73BB8B178484A424852F82C
:10D20000213000681B1A42F82130FFF730B8B1789E
:10D21000424A3D4B52F821001B68434342F82130FB
:10D22000FFF725B8B1783D4A374852F821300068F9
:10D2300093FBF0F342F82130FFF719B8B178374A81
:10D24000314B52F82140186894FBF0F300FB134374
:10D2500042F82130FFF70BB8B178304A2A4852F82B
:10D2600021300068034042F82130FFF700B8B17860
:10D270002A4A254852F821300068034342F82130F9
:10D28000FEF7F5BFB178254A1F4852F821300068F3
:10D29000434042F82130FEF7EABF1B4BB1781B68D0
:10D2A0001E4ADB4342F82130FEF7E1BF164BB2784D
:10D2B00019681A4B43F82210FEF7D9BFB178174A04
:10D2C000114B52F821001C6842F821401860FEF70B
:10D2D000CEBF124BB27853F822200B4B1B6864E789
:10D2E00003230B70FEF7C3BF7178074B084A0B2965
:10D2F00000F28780DFE801F014242B323A444B52CD
:10D30000595F646DBCC6FF1F5CD0FF1F78D0FF1F44
:10D31000E4CEFF1F7ACEFF1FE8CEFF1F88D0FF1F8D
:10D32000B0789E4951F820101868014419601B68B4
:10D33000002B69D1136843F008031360FEF797BF11
:10D34000B4789648196850F82400091AEEE7934912
:10D35000B07851F8200019684143E7E7B4788F4866
:10D36000196850F8240091FBF0F1DFE78B49B078A1
:10D370001C6851F8200094FBF0F100FB1141D5E747
:10D38000B078864951F8201018680140CEE7B0788F
:10D39000824951F8201018680143C7E7B0787F49E7
:10D3A00051F8201018684140C0E7B0787B4951F827
:10D3B0002010C943BAE7B078784951F82010B5E792
:10D3C000B07876491D6851F820401C6041F8205023
:10D3D000ADE77249B07851F82000196888421168A9
:10D3E00005DA21F0030141F0040111609FE70BBF52
:10D3F00021F0060121F0050141F0010141F0020197
:10D40000F3E70321297092E7136823F00803136000
:10D41000FEF72DBF73780B2B00F28680DFE803F058
:10D4200006111C2733414C57626B737EB1785B4AFF
:10D430005B4852F821300068034442F82130FEF77F
:10D4400016BFB178554A564852F8213000681B1A69
:10D4500042F82130FEF70BBFB178504A504B52F8DA
:10D4600021001B68434342F82130FEF700BFB1782A
:10D470004A4A4B4852F82130006893FBF0F342F8D7
:10D480002130FEF7F4BEB178444A454B52F82140B2
:10D49000186894FBF0F300FB134342F82130FEF7C9
:10D4A000E6BEB1783D4A3E4852F82130006803405C
:10D4B00042F82130FEF7DBBEB178384A384852F8DE
:10D4C00021300068034342F82130FEF7D0BEB17826
:10D4D000324A334852F821300068434042F8213044
:10D4E000FEF7C5BE2E4BB1781B682C4ADB4342F8D1
:10D4F0002130FEF7BCBE2A4BB2781968274B43F89F
:10D500002210FEF7B4BEB178244A254B52F8210010
:10D510001C6842F821401860FEF7A9BE1F4BB27884
:10D5200053F822201E4BD9E603230B70FEF79FBE53
:10D5300073780B2B00F29480DFE803F006101A24B6
:10D5400034414B555F68707B154AB178134B53F8E3
:10D55000213011680B441360FEF789BE104AB07881
:10D560000E49136851F820105B1A1360FEF77FBE56
:10D570000B4A0A4BB17853F8211013684B431360E0
:10D58000FEF775BE064AB0780449136851F82010BA
:10D5900093FBF1F31360FEF76ABE00BF88D0FF1F54
:10D5A00078D0FF1FB94ABA4BB178106853F82110F0
:10D5B00090FBF1F301FB13031360FEF758BEB34A6F
:10D5C000B178B34B53F8213011680B401360FEF76C
:10D5D0004EBEAE4AB178AE4B53F8213011680B43C2
:10D5E0001360FEF744BEA94AB178A94B53F8213025
:10D5F00011684B401360FEF73ABEB278A44B53F863
:10D600002230A24ADB431360FEF731BEA04BB27852
:10D6100053F822209D4B1A60FEF729BEB1789C4A30
:10D620009A4B52F821001C6842F821401860FEF71E
:10D630001EBE974BB27853F82220944B1B689A4237
:10D64000FFF6B6AD934A13680BBF23F0060323F031
:10D65000050343F0010343F002031360FEF707BE26
:10D6600003230B70FEF703BEB178894A52F82130CC
:10D67000184442F82100FEF7FABDB178844A52F806
:10D680002130181A42F82100FEF7F1BDB178804A26
:10D6900052F82130584342F82100FEF7E8BDB17836
:10D6A0007B4A52F8213093FBF0F042F82100FEF75C
:10D6B000DEBDB178764A52F8214094FBF0F300FBCE
:10D6C000134042F82100FEF7D2BDB178704A52F8FB
:10D6D0002130184042F82100FEF7C9BDB1786C4AEC
:10D6E00052F82130184342F82100FEF7C0BDB1784E
:10D6F000674A52F82130584042F82100FEF7B7BD82
:10D70000B178634A52F82130DB4342F82130FEF70A
:10D71000AEBDB2785E4B43F82200FEF7A8BDB278EA
:10D720005B4B53F8223098428AE703230B70FEF7D5
:10D730009EBD594B1B68C6F80330FEF7DBF9FEF7B8
:10D7400096BD524B1B68B370534B1B68C6F8033031
:10D75000FEF7D0F9FEF78BBDFCF712FF4F4B01220D
:10D7600083F8C020D6F80320C3F8C420FEF77FBD9D
:10D770007178474A52F82130013B002B42F82130A2
:10D780007EF775AD454BC3F8C400FEF770BD424B44
:10D790001B68C6F80330FEF74FF83C4B1B68A370BC
:10D7A0003D4B1B68C4F80330FEF798F8FEF75FBDE9
:10D7B000364B1B68B370384B1B68C6F80330FEF756
:10D7C0003BF8FEF754BD314B1B78B370FEF756BDE6
:10D7D0002E4B1B68B370FCF7FDFEFEF748BD2B4BCC
:10D7E0001B68B370FDF706FAFEF741BD274B1B68B7
:10D7F000B370294B1B68C6F80330FCF7EBFEFEF74D
:10D8000036BD224B1B68FF2B3EF631AD204A52F845
:10D810002320214B4A601A601E4B2AB91A6842F035
:10D8200008021A60FEF723BD1A6822F008021A6087
:10D83000FEF71DBD194BD3F8C820072A3EF617ADD9
:10D8400071780C293EF613ADDFE811F00D002A00C7
:10D850003C004E006000720085009700A900BB00EC
:10D86000CD00DF00F1000B4909680C077EF5FFAC25
:10D87000511C03EB8202C3F8C810D3F8C410C2F8DD
:10D88000E410C3F8C400FEF7F2BC00BF78D0FF1F5D
:10D8900088D0FF1FE4CEFF1F5CD0FF1FBCC6FF1F58
:10D8A000CE49096809073EF5E2AC511C03EB820240
:10D8B000C3F8C810D3F8C410C2F8E410C3F8C40009
:10D8C000FEF7D5BCC5490968CF077EF5D0AC511C21
:10D8D00003EB8202C3F8C810D3F8C410C2F8E410F6
:10D8E000C3F8C400FEF7C3BCBC490968CE073EF5C7
:10D8F000BEAC511C03EB8202C3F8C810D3F8C410AD
:10D90000C2F8E410C3F8C400FEF7B1BCB34909681B
:10D910004D077EF5ACAC511C03EB8202C3F8C81076
:10D92000D3F8C410C2F8E410C3F8C400FEF79FBCDB
:10D93000AA49096811F0050F3EF499AC511C03EB9C
:10D940008202C3F8C810D3F8C410C2F8E410C3F8B8
:10D95000C400FEF78CBCA14909688C077EF587AC32
:10D96000511C03EB8202C3F8C810D3F8C410C2F8EC
:10D97000E410C3F8C400FEF77ABC98490968890727
:10D980003EF475AC511C03EB8202C3F8C810D3F807
:10D99000C410C2F8E410C3F8C400FEF768BC8F4995
:10D9A0000968CF067EF563AC511C03EB8202C3F815
:10D9B000C810D3F8C410C2F8E410C3F8C400FEF7CE
:10D9C00056BC864909688E067EF551AC511C03EBA6
:10D9D0008202C3F8C810D3F8C410C2F8E410C3F828
:10D9E000C400FEF744BC7D4909684D067EF53FAC96
:10D9F000511C03EB8202C3F8C810D3F8C410C2F85C
:10DA0000E410C3F8C400FEF732BC744909680C0680
:10DA10007EF52DAC511C03EB8202C3F8C810D3F87D
:10DA2000C410C2F8E410C3F8C400FEF720BC6B4970
:10DA30000968C9057EF51BAC511C03EB8202C3F8D3
:10DA4000C810D3F8C410C2F8E410C3F8C400FEF73D
:10DA50000EBC00F0B5FEFEF70ABC00F0D1FEFEF7EA
:10DA600006BC00F0E2FEFEF702BC00F0DFFEFEF7AF
:10DA7000FEBB00F0DCFEFEF7FABB00F0D9FEFEF7BD
:10DA8000F6BB73782BB1012B09D003230B70FEF783
:10DA9000EEBB534B012283F8C020FEF7E8BB40F2F7
:10DAA000FE7290423EF606AC4D4A82F8C030C2F893
:10DAB000C400FEF7DCBB4A4B022283F8C020FEF70D
:10DAC000D6BB484B1B7D9B070CD440F2FE7398429B
:10DAD0003EF6F0AB424B042283F8C020C3F82C0181
:10DAE000FEF7C5BB08230B70FEF7C1BB3C4B002201
:10DAF00083F8C020FEF7BBBB3B4B3C4D01221A70A4
:10DB0000384B9978297040F2FE71884226D81B7DE7
:10DB100013EA020422D16946FBF73CFA9DF8003073
:10DB20006B709DF80130AB709DF80230EB709DF882
:10DB300006302B719DF805306B719DF80430AB7188
:10DB40009DF80330EB712C720123E95C2A7A0133D2
:10DB50000A44082B2A72F8D1FEF789BB0123002260
:10DB6000EA540133082BFBD12B782B72FEF77FBBD5
:10DB70001D4B01221A701B4B1C4A9B7813701C4BC7
:10DB8000196800230139013311F8010FD054082B13
:10DB9000F9D1FEF76CBB0422CA714B7156220B23DC
:10DBA0008A710B71FEF763BB0F4B124801221A708A
:10DBB0000C4B0E4A9B781370002301331918082B65
:10DBC00011F8091CD154F8D1FEF751BB7378032B1F
:10DBD0003EF64DABDFE803F0101E2C31E4CEFF1F04
:10DBE000BCC6FF1F0CC0FF1F60D0FF1F61D0FF1F0E
:10DBF00008C0FF1F00800000854B93F8C020CA7149
:10DC000093F8CC20D3F82C318A711A0A4A710B711F
:10DC1000FEF72DBB7E4B93F8C020CA7193F8CC2041
:10DC2000D3F8C4308A711A0A4A710B71FEF71FBB10
:10DC3000784B1B684B60FEF71ABB774B1B684B6039
:10DC4000FEF715BB7378002B7EF411ABB378002B75
:10DC50007EF40DAB40F2D24398427EF408AB002133
:10DC600040F2FF70FBF770FAFBF7D5F90120FAF7E5
:10DC700027FEFEF7FCBA7278684B9AB91A70684AA8
:10DC8000E3781370624A92F83011664A117066495F
:10DC900000220A7065490A70654A11780B431370B7
:10DCA000FEF7E5BA0122E9E70422694640F2FB707B
:10DCB000FBF73CFB009BD4F803209A4206BF0123EC
:10DCC0006B606E60FEF7D3BAA3782A2B07D10422CB
:10DCD000584940F2FB70FBF796FAFEF7C8BA0323E7
:10DCE0000B70FEF7C4BA7378032B47D8DFE803F054
:10DCF0001B023442464CD4F83411002204F59C73C4
:10DD00008A423EF4B4AA53F82250854202F101053A
:10DD100020D103EB8503043B01398A4214D3C4F8B4
:10DD20003411FEF7A4BA3A4BD3F83421092A9DBF27
:10DD3000511CC3F8341103EB8203092394BFC3F8C9
:10DD400038012B70FEF793BA53F8040F43F8040C14
:10DD50000132E2E72A46D3E72D4A0023C2F83431E4
:10DD6000194602F59C7242F8231001330A2BFAD1AE
:10DD7000FEF77DBA0A234B60FEF779BA03230B70D6
:10DD8000FEF775BA7378812B7EF494AAB378922B40
:10DD90007EF490AAB379A32B7EF48CAA7379B42B6A
:10DDA0007EF488AA3379C52B7EF484AAF378D62B27
:10DDB0007EF480AAFBF759F8FAF7A6FC0446FAF7B6
:10DDC000A3FC001B0028B8BF4042B0F57A7FF6DB09
:10DDD000FAF774FD184B00221A604FF0FF32C3F8B7
:10DDE0007021C3F87022C3F87421C3F87422C3F8F9
:10DDF0007821C3F87822C3F87C21C3F87C220F4B2A
:10DE00000F4A1A600120FAF75BFDFEF730BA00BF37
:10DE1000BCC6FF1F5CD0FF1F78D0FF1F18CDFF1FAF
:10DE200044CDFF1F70CEFF1F43CDFF1FA9CEFF1FA4
:10DE300019CDFF1FDFCEFF1F10E000E000C0FF1F65
:10DE400078563412344B2DE9F04100241C60334BDA
:10DE5000334D1C60334BDFF8E480334FC5F8C440CA
:10DE60001C6085F8CC406601F6B246F00601002041
:10DE7000FBF784FE46F00C0148F824000020FBF775
:10DE80007DFE47F824000134032CECD1274BD97ACE
:10DE9000C1F10801C9B20020FCF7ECF8244A0023C4
:10DEA0001946174642F823100133B3F5807FF9D1A4
:10DEB000204CA37E7BB1204E0C25002405F20C677C
:10DEC00029193819042231440434FBF72FFA0C2C99
:10DED000F6D10C35F1E7E37E73B194F824100020FD
:10DEE000FBF7A0FC637DABB1FAF784FF90B101238F
:10DEF00085F8C030BDE8F0814FF4A766A6F5A761AC
:10DF00003046042239440436FBF710FAB6F5C36FE5
:10DF1000F4D1E2E70023EBE75CD0FF1F78D0FF1FCE
:10DF2000BCC6FF1FE4CEFF1F7CD0FF1FB8CDFF1F74
:10DF300088D0FF1F0CC0FF1FE8CEFF1F88D4FF1F33
:10DF4000F7B50F4C07460E4694E803008DE8030032
:10DF50000C49C1F803300C4B8A7000220F704E70D0
:10DF60001A70FDF7A3FF094A217882F861119DE834
:10DF70000300636884E80300184603B0F0BD00BFE7
:10DF800070D0FF1FDCCEFF1F6BD0FF1FBCC6FF1F72
:10DF9000F7B504461F4A63781370A3785370E3788B
:10DFA00093702379937163795371A3791A4D137127
:10DFB000E379D3700E4695E80300184B00221A70DF
:10DFC0008DE80300FDF772FF154B1A786F462B465C
:10DFD0009AB9327072702A78B2706A78F270EA79FF
:10DFE0003271AA7972716A79B2712A79F27197E8FD
:10DFF000030083E8030003B0F0BD012AF7D109480C
:10E00000721EF11D10F8014F02F8014F8A42F9D13A
:10E01000EDE700BFDCCEFF1F70D0FF1F6BD0FF1FEE
:10E0200060D0FF1F61D0FF1F014B93F86101704763
:10E03000BCC6FF1F2DE9F043994B9A4C1B788FB05B
:10E040006BB1994B1B78063BDBB2192B04D8974A6E
:10E0500022FA03F3D90702D4002384F8303194F86C
:10E060003031934E5A1E012A51D89249012BCA6869
:10E07000079214BF082307238DF81830327894F8DC
:10E0800062318DF8193000238DF81A30002A33D10F
:10E090008B688DF82030884B8DF8272019788DF803
:10E0A000211059788DF82210D9798DF8231099799B
:10E0B0008DF8241059791B798DF825108DF82630AC
:10E0C00006A801F0F3FD002800F029837B4B1A78A5
:10E0D0009846002A00F01E81794B7A4F1B78013B4D
:10E0E000062B00F21381DFE813F0F100F100580174
:10E0F0001101110111017F01012AE1D1724801339F
:10E1000006AA1A44195CD171082BF8D1D8E7032B61
:10E110003DD1337883BBDFF89C81674F98F80200CC
:10E1200098F801503B7805441D447B781D44FB79E9
:10E130001D44BB791D447B791D443B791D44FAF78E
:10E140001DFB98F80100FAF719FB3878FAF716FB6F
:10E150007878FAF713FBF879FAF710FBB879FAF741
:10E160000DFB7879FAF70AFB3879EDB2FAF706FB7E
:10E170002846FAF703FBA9E7012BA7D1524F002548
:10E18000785D0135FAF7FAFA092DF9D19EE7042BEB
:10E190002BD1484FDFF82081B8787D780023012209
:10E1A0000544154488F8013088F80020C8F8043088
:10E1B000FAF7E4FA7878FAF7E1FA98F80000FAF753
:10E1C000DDFA98F80100FAF7D9FA98F80700FAF79B
:10E1D000D5FA98F80600FAF7D1FA98F80500FAF798
:10E1E000CDFAEDB298F80400C0E7072B37D13378A9
:10E1F00053BB304B9F7893F801802F4B8DF8007004
:10E200001D785878D9798DF8025047443D449A7961
:10E210008DF80300284493F805C08DF804100144DC
:10E2200093F804E08DF805200A440CEB02037344D4
:10E230008DF801808DF806C08DF807E08DF8083064
:10E240006846FAF70FFE41E7012BF9D11E4900237A
:10E250005A5C0DF803200133092BF9D1F0E7082BA4
:10E260007FF434AF144A1349002301205370107017
:10E2700053608A7849788DF800200A4402448DF86A
:10E2800001108DF802008DF803308DF804308DF800
:10E2900005308DF806308DF807308DF80820CFE76F
:10E2A0006AD0FF1FBCC6FF1FDCCEFF1F1102000299
:10E2B00060D0FF1F0CC0FF1F70D0FF1FA9CEFF1F33
:10E2C00070CEFF1F43CDFF1F61D0FF1FB14A3978C9
:10E2D00093688DF8303080238DF831308A238DF8A3
:10E2E000323000238DF833308DF834308DF83530EE
:10E2F0008DF836108DF8293007218DF82A300AA8BC
:10E30000D3688DF828100B9301F0D0FC00233B70EC
:10E3100088F80030002384F83031337094F860318D
:10E3200013B10120FAF7CCFA06A801F04BFC06461F
:10E33000002800F04781984B9DF820201A709DF826
:10E3400021205A709DF822209A709DF823209A71FE
:10E350009DF824205A719DF825201A719DF82620D9
:10E36000DA709DF8193084F86231FAF7CDF98B4BE9
:10E3700018608B4B00221A709DF81830072B0CBFC9
:10E380000123022384F8303194F8C0305A1E012A48
:10E390004AD9052B48D0012247E0DFF8F8913B78B5
:10E3A00099F8020099F8015005440A351D44FAF71E
:10E3B000E5F999F80100FAF7E1F98020FAF7DEF9BA
:10E3C0008A20FAF7DBF90020FAF7D8F90020FAF7EB
:10E3D000D5F90020FAF7D2F9EDB23878FAF7CEF98C
:10E3E0002846FAF7CBF991E76A4A507893788DF886
:10E3F0000C303A788DF80D00802103448DF80E1012
:10E400000A338A218DF80F101344002103A88DF8D8
:10E4100010108DF811108DF812108DF813208DF852
:10E420001430FAF71FFD71E700225E4B1A7094F862
:10E43000C030042B04D1584B19780A0640F1728180
:10E4400094F83021082A04D840F25113D340DF0752
:10E4500001D4FDF72BFD94F83031092B74D1FAF774
:10E4600053F9D4F8D830504DC01A00282A68B8BFE4
:10E470004042904209D94D4B1A78012A04BF02222A
:10E480001A70FAF741F9C4F8D800FAF73DF9D4F850
:10E49000DC306A68C01A0028B8BF4042904209D9EF
:10E4A000424B5A78012A04BF02225A70FAF72CF91B
:10E4B000C4F8DC00FAF728F9D4F8E030AA68C01AEA
:10E4C0000028B8BF4042904209D9384B9A78012AB7
:10E4D00004BF02229A70FAF717F9C4F8E000237813
:10E4E00093B3637883BB314A31481D46D15C02291E
:10E4F00040F00C8150F823104E1C00F006812D4A8C
:10E5000084F828311268C4F80C212B4A1268C4F828
:10E510001021D4F8C420C4F81421284AC4F8C41027
:10E520001268C4F8182194F8CC20C4F81C210023E8
:10E53000D4F80821C4F8202184F8CC30D4F8042180
:10E54000C4F824210123637094F83031092B06D1DB
:10E5500094F8C020022A04BF052284F8C020D4F811
:10E560003421002A00F0DB80092B40F0D88094F899
:10E57000C030012B40F0D380D4F8C41010480023E1
:10E5800050F823508D4240F0C680052384F8C030F7
:10E59000C5E000BF0CC0FF1FDCCEFF1F60CEFF1F19
:10E5A00008CDFF1F6BD0FF1F28CEFF1F7ACEFF1FA5
:10E5B000C0C6FF1F5CD0FF1F78D0FF1FE4CEFF1F37
:10E5C000F4C7FF1F03A8FAF7F1F8054600284ED05C
:10E5D000FAF704F908B184F8636194F863219DF8AF
:10E5E0000C10531CDBB22244092B84F8633182F8EF
:10E5F00064117FF41CAF614A94F8641152780023CF
:10E60000914284F863317FF412AF5D495A5C013363
:10E610001644082BF6B2F9D194F86C31B34222D1EA
:10E62000584B94F865211A7094F866215A7094F842
:10E6300067219A7094F868219A7194F869215A7147
:10E6400094F86A211A7194F86B21DA70FAF75CF881
:10E650004D4B4E4A186000231370032284F830217A
:10E6600084F8633190E6042384F83031DFE60AAEA3
:10E670003046FAF7E4FB48B32B46F25C013315440D
:10E68000082BEDB2F9D19DF83020AA42ECD13D4BD8
:10E690009DF829201A709DF82A205A709DF82B2089
:10E6A0009A709DF82C209A719DF82D205A719DF832
:10E6B0002E201A719DF82F20DA70FAF725F8324BC8
:10E6C0001860324B00221A7007235BE694F8C030C2
:10E6D000013B012B3FF6ABAED4F8C42040F2FE73F1
:10E6E0009A420ED8FAF786FB58B1D4F8C4002549EF
:10E6F000431CC4F8C430FAF74DFC092384F83031C8
:10E7000049E6002384F8C03091E6D55401332F2B1D
:10E710007FF4ECAE18E701339A427FF431AF0FB0CB
:10E72000BDE8F08394F83001082804D840F2511273
:10E73000C240D207F3D4164DD3F80330D4F82C01DD
:10E740006B6040F2FE739842697012D80D49FAF777
:10E7500031FD0C49D4F82C01FAF79EFC38B1D4F8FD
:10E760002C310133C4F82C3165232B70D7E70723F4
:10E77000FBE707232B70002308E700BF0CC0FF1F37
:10E7800020C8FF1FDCCEFF1F68CEFF1F6FCEFF1F0C
:10E7900070D0FF1F704710B5074CF9F7B5FF23681D
:10E7A000C01AB0F5FA7F05D9044B2022DA60F9F7D8
:10E7B000ABFF206010BD00BF94D4FF1F00F00F40DE
:10E7C00007B50D4B5A782AB1012A0AD00B4B032208
:10E7D0001A700EE0D978987803B05DF804EBFBF777
:10E7E000B7BD1A799878DB78009300231946FBF7B8
:10E7F00013FE03B05DF804FBDCCEFF1F70D0FF1FDB
:10E80000064B5A7832B9D3F80310054B01B90122EF
:10E810001A7070470322034BFAE700BFDCCEFF1FDC
:10E820003CCDFF1F70D0FF1F704770477047704787
:10E83000704770472DE9F04F9E4C237885B033B96F
:10E840006FF000436360A360E36001232370257CC5
:10E85000DFF8A0824DB9E8B2FAF76CF908F80500C4
:10E860000135082DF7D101232374DFF88CA2924FD4
:10E87000272500264FF00209F0B2FAF75BF918F8E5
:10E880000630834216D0B31D08F806005AF823302C
:10E89000022B0AD0032B02D0012B0BD150B17B5D90
:10E8A000012B08BF07F8059004E018B97A5D012A2A
:10E8B00000D17B550136082E05F10105DCD17F4DD5
:10E8C000EB69C3B17E4E3778AFB9F9F71DFF7D4BC9
:10E8D0001B68C01A0028EB69B8BF404298420AD9A9
:10E8E0003846FBF795F80120FBF792F80220FBF77A
:10E8F0008FF8012333702B6AC3B1734E3778AFB9E9
:10E90000F9F702FF714B1B68C01A00282B6AB8BFC9
:10E91000404298420AD93846FBF77AF80120FBF7C3
:10E9200077F80220FBF774F801233370684D2B7BD6
:10E93000002B40F0B482F9F7E7FEE369C01A002823
:10E94000B8BF40420A2804DC624B1B69DF0700F1B4
:10E95000258294F82000002840F047810A21FAF728
:10E9600005FF074694F820005B4EFBF791F9002F56
:10E9700040D194F82010490141F0080101F0E8016C
:10E980003846FAF7F3FEA8BBF9F7BEFE94F820204C
:10E9900004EB820305EB42115B68B1F81CE0C01A7E
:10E9A00000284FF00A03B8BF404203FB0EF3984221
:10E9B00008DD897A1046F9F791FF94F8203001219B
:10E9C000464AD15494F8200087EAE77856F8303068
:10E9D000A8EBE77898452BD2FBF74CFC94F8203055
:10E9E00006EBC306727982422BD100211846FBF751
:10E9F0000FFC26E094F8200087EAE77256F83030E2
:10EA0000A2EBE7729A4235BF06EBC00305EB401359
:10EA10001979597AF9F762FF94F82080F9F774FEB2
:10EA200004EB880894F82030C8F804000021C7E7F8
:10EA3000FBF720FC94F8203006EBC306717988427E
:10EA4000D4D194F82000264B03440193254B034472
:10EA50000093254B002203EB80031146FBF7F0FCEB
:10EA600094F8200005EB40139B69BBB1FAF780F9DD
:10EA7000A0B194F8200005EB40139B6998450DD98F
:10EA8000FAF7C6FF94F82030184A0121D1540F3309
:10EA9000094AD15C012904BF0221D15477B394F80B
:10EAA0002060134B9B5DABBBF9F72EFE04EB860693
:10EAB000706255E02CC8FF1F7ACEFF1F0CC0FF1FED
:10EAC0006FCEFF1F68CEFF1F08CDFF1F60CEFF1F58
:10EAD000B8CDFF1FC0F00F4024CDFF1F71CEFF1F28
:10EAE000B3CDFF1F20CDFF1F48CDFF1FB0CDFF1FAF
:10EAF00074CEFF1F3DC8FF1F28CEFF1F94F82010C3
:10EB0000490141F0080101F0E8013846FAF72EFE0C
:10EB10000028C4D194F8203005EB4312D28912B9F1
:10EB2000AA4AD35CE3B1F9F7EFFD94F8202004EB97
:10EB300082035B6AC01A05EB42130028D9894FF0A3
:10EB40000A03B8BF40424B43984209DDA04EB35C74
:10EB500033B91046FBF7E0FC94F820300122F25460
:10EB600094F8202051016B185B69002B3DD0994B24
:10EB70009E5C9846CEBBC7B341F0020101F0E201B2
:10EB80003046FAF7FBFF074694F8200001F05CF9E5
:10EB900094F8201005EB4113381A5B69002883EACA
:10EBA000E372B8BF4042A2EBE37290421DDD002B3E
:10EBB00040F31E810846FAF72BFF94F8203005EB4E
:10EBC00043139B7F002B40F0EC8094F82030824A66
:10EBD0001533D15C012901D10221D15494F82000D0
:10EBE000012308F8003000F0A1FE0020FAF7A1FD93
:10EBF00094F830308DF8080003F0F803C60748BFDA
:10EC000043F0010384F83030450748BF94F83030B2
:10EC1000DFF8D8A144BF43F0020384F83030C006C7
:10EC200048BF94F830309AF800C044BF43F0040362
:10EC300084F83030694B94F830001978684B1E78AE
:10EC4000684B1D78684B93F8009000231F469E4642
:10EC500098461A464CFA02FB1BF0010F40F0028165
:10EC60000132032AF6D1B8F1000F01D08AF800C0B2
:10EC7000BEF1000F01D0594A11700FB1584A1670F9
:10EC80000BB1584B1D70C10709D594F83130DA0724
:10EC900005D4514BDA78012A04BF0222DA708307C7
:10ECA00009D594F831309F0705D44B4B1A79012AC6
:10ECB00004BF02221A71460709D594F831305D0766
:10ECC00005D4454B5A79012A04BF02225A7104AA7D
:10ECD00094F8201084F831000323B1FBF3F31344BC
:10ECE00013F9083C002B49DA490141F0160103AA47
:10ECF00001F0F6010020FAF722FD9DF80E305806CB
:10ED00000AD594F8202002201B2110FB0212324960
:10ED10008D5C012D08BF885419060AD594F820206F
:10ED20002D490E3211F81200012804BF022001F80B
:10ED30001200DA060AD594F8202002201B2110FBCD
:10ED4000021225498D5C012D08BF88549B060AD507
:10ED500094F82030204A0E3312F81310012904BF12
:10ED6000022102F8131094F82010490141F0160115
:10ED700003AA01F0F6010020FAF71CFC94F8200029
:10ED800000F002F994F820300133DBB2032B88BF86
:10ED9000002384F82030F9F7B7FCE06105B0BDE846
:10EDA000F08F94F8202005EB461305EB42129B7F71
:10EDB000927F9A4205D13046FAF72AFEF0B200F06F
:10EDC000B5FD0136032EECD1FFE600BF74CEFF1F68
:10EDD00077CEFF1F40CDFF1F7ACEFF1F19CDFF1F3B
:10EDE00043CDFF1FA9CEFF1F18CDFF1F44CDFF1F2E
:10EDF00002223046FAF7D0FC94F82010490141F085
:10EE0000080101F0E8013046FAF77CFC94F8203064
:10EE100005EB43139B7F002B3FF4E0AE94F82020DA
:10EE200005EB461305EB42129B7F927F9A4210D16D
:10EE3000F7B2022239460020FAF7AEFC790141F020
:10EE40000801002001F0E801FAF75CFC384600F008
:10EE50006DFD0136032EE1D1C0E601231D461F469C
:10EE60009E46FDE640FA02FB1BF0010F3FF4F8AEB0
:10EE700041FA02FB1BF0010F7FF4F2AE0123934035
:10EE80005BB219431E43C9B2F6B2B9F1000FE4D127
:10EE90000123CC461D461F469E469846E0E60022CA
:10EEA000354E364B84F820201046019600931146CB
:10EEB000334BFBF7C5FA94F820003356314E002B44
:10EEC00004EB000393F832301CDB022B01D1335CDE
:10EED00083B105EB4015697AF9F700FD94F820003D
:10EEE000FBF724FB94F82030E218022182F832105C
:10EEF0000022F25494F82050F9F706FC04EB850444
:10EF000060604BE7012B1DD194F82030F35C002B9F
:10EF10003FF444AF94F8200005EB4013997AF9F7D9
:10EF2000DDFC94F8200005EB4015AB7AF3B9FBF754
:10EF3000F3FA94F820301C44012284F83220002295
:10EF4000F2542BE7F9F7E0FB94F8202004EB82035E
:10EF500005EB42125B68928BC01A00284FF00A033F
:10EF6000B8BF404253439842CEDDD3E7335C002B19
:10EF7000DFD0FBF7DBFADCE7B3CDFF1F20CDFF1FAF
:10EF800048CDFF1F6CCEFF1F2DE9F04F46014FFA11
:10EF900086FB85B04BF07C01044603AA01F0FC011E
:10EFA0000020FAF7CCFB4FEA44099DF90EA0A64DCC
:10EFB0000222012303FA09F302FA09F20AEA020221
:10EFC0000AEA030AAB19D2B21B7A009203F07F0758
:10EFD0001B065FFA8AFA4FF0000013D5F9F7AAFD75
:10EFE000B0FA80F35B09791E009A072900F28A8241
:10EFF000DFE811F00E000E000E000E008B028B02F7
:10F000008B028B02F9F796FD031C18BF0123EAE778
:10F010008E490B5D88460F2B00F27482DFE813F0F7
:10F020007202100054007D008F00B800CF00F20083
:10F030001E016701CF01D40172021D02480226029F
:10F040004FF0000A5FFA8AFB5C4507D0AA19927F4D
:10F0500082B305EB4A11897F91422BD14FEA4B19BC
:10F060004FFA89F949F0140103AA01F0F4010020D4
:10F07000FAF765FB49F00609754B9DF80D2043F83A
:10F080002A205FFA89F949460020FAF76FFB714B95
:10F09000022243F82A0059460020FAF77DFB40F28D
:10F0A000FF7249460020FAF7AAFA032259460020C7
:10F0B000FAF795FB0AF1010ABAF1030FC2D1023F38
:10F0C000012F38D8022337E008EB840321465A6821
:10F0D00002F0040242F001020020FAF780FB002750
:10F0E000B9462E445FFA89F39C4205D0B37F53B1F1
:10F0F0007A19927F9A4206D147F008017A59C9B22B
:10F100000020FAF77CFA09F10109B9F1030F07F1C0
:10F110002007E7D108F80490F4E1BAF1000F00F0FD
:10F12000F1814BF0020101F0E2010020FAF726FD27
:10F13000494B43F82400042308F80430E2E108EBCB
:10F14000840321465A6802F0040242F002020020C1
:10F15000FAF745FB0027B9462E445FFA89F39C4233
:10F1600005D0B37F5BB17A19927F9A4207D17A5961
:10F1700047F008015242C9B20020FAF740FA09F1FB
:10F180000109B9F1030F07F12007E6D10523D3E701
:10F19000002A00F0B78100272E44FBB2A34206D01C
:10F1A000B37F3BB105EB4712927F9A4202D13846BA
:10F1B000FAF72EFC0137032FEFD10623BCE7032219
:10F1C00021460020FAF70BFBDFF87C90002735443E
:10F1D000F9B28C4205D0AB7F6BB199F81E209A42F0
:10F1E00009D1490141F00801D9F8042001F0E801F2
:10F1F0000020FAF704FA0137032F09F12009E7D1BB
:10F20000072399E7002A40F07D810F4F914635444E
:10F210005FFA89F1A14204D0AB7F63B1BA7F9A4211
:10F2200009D17A68490141F00801524201F0E80130
:10F230000020FAF7E4F909F10109B9F1030F07F128
:10F240002007E5D1082377E7B8CDFF1F64C8FF1F6B
:10F2500068C8FF1F74C8FF1F0CCDFF1F002A00F0F5
:10F2600051814BF0020101F0E2010020FAF786FC27
:10F27000BA4A52F8243000271B1A42F82430834639
:10F28000B946AB195FFA89F6B44205D09A7F2AB322
:10F290007919897F914221D14FFA87FA00224AF0E9
:10F2A00008011046C9B20093FAF7A9F903223146C2
:10F2B0000020FAF794FA7A194AF006015268C9B2A6
:10F2C0000020FAF79CF95A46F9B20020FAF7A9F99A
:10F2D000002231461046FAF75FFA009B09F1010956
:10F2E000B9F1030F07F12007CCD1092324E700204F
:10F2F000FAF71FFA40FA09F0C10740F103814FF015
:10F300000009AB19CA4600935FFA8AF39C4207D002
:10F31000009A927F0AB309EB0501897F91421CD1C3
:10F320004FFA89FB00224BF008011046C9B2019345
:10F33000FAF765F9019B022219460020FAF72CFA28
:10F3400000224BF002011046C9B2FAF76AF9002216
:10F350005FFA89F11046FAF764F90AF1010ABAF185
:10F36000030F09F12009CFD1033F012F7CD8DFF82B
:10F37000F4A14FF0000935445FFA89F7BC4205D08B
:10F38000AB7F9BB19AF81E209A420FD102223946D8
:10F390000020FAF701FADAF80420790141F00801B7
:10F3A000524201F0E8010020FAF729F909F10109B8
:10F3B000B9F1030F0AF1200ADED10A23BCE6002AC4
:10F3C00000F0A0800B23B7E6002A40F09B804BF0B2
:10F3D0000201104601F0E2010092FAF7CFFB009A19
:10F3E0008146174605EB060AF9B28C4207D09AF817
:10F3F0001E306BB105EB4712927F9A4208D149014A
:10F4000041F00801002201F0E8011046FAF7F7F890
:10F410000137032FE8D100272E44022399FBF3F98B
:10F420005FFA87FA544506D0B37F8BB105EB4712DC
:10F43000927F9A420CD14FEA4A114A4601F0E0010C
:10F440000020FAF7EEF8002251461046FAF7A4F928
:10F450000137032FE4D10D236EE60020FAF769F996
:10F4600040FA09F0C2074DD50E2365E64FF00009BA
:10F470002E445FFA89F7BC4206D0B37F93B105EB07
:10F480004912927F9A420DD1022239460020FAF7A2
:10F4900083F9790141F00801002201F0E8011046EA
:10F4A000FAF7ADF809F10109B9F1030FE1D1DBE792
:10F4B000DFF8B4A000273B46AAF10C0B5FFA87F9EE
:10F4C0004C4507D0AA19927FCAB105EB4711897F35
:10F4D000914214D14FEA491141F006015AF8272010
:10F4E000009301F0E6010020FAF789F81BF82720C5
:10F4F00049460020FAF773F9009B08F807300137F6
:10F50000032FDBD105B0BDE8F08F1548015D8046C3
:10F510000F29F7D801A050F821F000BF05F5000031
:10F520006DF50000E9F5000043F6000063F6000009
:10F53000BFF6000005F50000D5F6000005F5000057
:10F5400005F500008FF70000ABF7000031F7000071
:10F5500029F80000E9F80000A5F800000CCDFF1F15
:10F5600064C8FF1FB8CDFF1F74C8FF1F4FF0000A0B
:10F570005FFA8AFB5C4507D0AA19927F42B305EB7C
:10F580004A11897F914223D14FEA4B194FFA89F9E9
:10F5900049F0140103AA01F0F4010020FAF7CFF8B2
:10F5A000BE4B9DF80D2043F82A2059460222002028
:10F5B000FAF7F2F849F0060140F2FF7201F0E601B5
:10F5C0000020FAF71CF8032259460020FAF707F941
:10F5D0000AF1010ABAF1030FCAD1062F3FF472AD46
:10F5E000082F7FF4A8AD6DE5062F26D108EB840324
:10F5F0005A6802F0040242F0010221460020FAF7A4
:10F60000EEF80027B9462E445FFA89F39C4205D0F4
:10F61000B37F53B17A19927F9A4206D147F008011D
:10F620007A59C9B20020F9F7EAFF09F10109B9F1E5
:10F63000030F07F12007E7D16CE5082FE1D1032282
:10F64000DBE77A1F012A07D8BAF1000F04D0062F92
:10F650003FF471AD0F236FE5002B3FF453AF0C2344
:10F660006AE5052F27D108EB84035A6802F00402EB
:10F6700042F0020221460020FAF7B1F80027B9460D
:10F680002E445FFA89F39C4205D0B37F5BB17A19AF
:10F69000927F9A4207D17A5947F008015242C9B283
:10F6A0000020F9F7ACFF09F10109B9F1030F07F1E7
:10F6B0002007E6D16AE5072FE0D10322DAE7791FB8
:10F6C000012903D812B1052FC4D1FBE4002B7FF42C
:10F6D00097AD17E7002B7FF415AF073F012F0AD92D
:10F6E00008EB84022146526802F0040242F0010253
:10F6F0001846FAF774F8DFF8A89100273544F9B2F4
:10F700008C4205D0AB7F6BB199F81E209A4209D18B
:10F71000490141F00801D9F8042001F0E801002076
:10F72000F9F76DFF0137032F09F12009E7D144E60E
:10F73000002B7FF4E7AE073F012F0AD908EB8402C4
:10F740002146526802F0040242F002021846FAF71B
:10F7500046F8DFF84C9100273544F9B28C4205D0C9
:10F76000AB7F73B199F81E209A420AD1D9F80420D0
:10F77000490141F00801524201F0E8010020F9F787
:10F780003EFF0137032F09F12009E6D115E6002BD2
:10F790003FF4B8AE4BF0020101F0E2010020FAF7AD
:10F7A000EDF908EB8403D8610CE6002B7FF4AAAED8
:10F7B0004BF00201184601F0E2010093FAF7DEF97E
:10F7C000009BAA19824653731F46994608EB840B87
:10F7D0005FFA89F39C4206D0AA19927FE2B17919A7
:10F7E000897F914218D17A1947F006015268009337
:10F7F000C9B20020F9F715FFDBF81C200221002018
:10F80000524492FBF1F2F9B2F9F70BFF009B002290
:10F8100019461046F9F7C0FF09F10109B9F1030FC4
:10F8200007F12007D4D116E60020F9F782FF40FA4D
:10F8300009F0C3077FF566AE0E23002708F80430F1
:10F84000B9462E445FFA89FA544505D0B37FEBB12F
:10F850007A19927F9A4219D14FFA87F8002248F01C
:10F8600008011046C9B2F9F7CAFE0222514600202B
:10F87000F9F792FF002248F002011046C9B2F9F7E9
:10F88000D0FE0022F9B21046F9F7CBFE09F10109CA
:10F89000B9F1030F07F12007D4D133E668C8FF1F81
:10F8A000B8CDFF1F4FF000092E445FFA89F7BC4224
:10F8B00006D0B37F93B105EB4912927F9A420DD1E6
:10F8C000022239460020F9F767FF790141F008016B
:10F8D000002201F0E8011046F9F791FE09F1010953
:10F8E000B9F1030FE1D1BFE5DFF82C9000272E44DA
:10F8F000F9B28C4206D0B37F4BB105EB4712927F31
:10F900009A4204D119F827200020F9F768FF01373F
:10F91000032FEDD100230FE468C8FF1F024B1A5CD0
:10F920000AB901221A54704764C8FF1F024B1A5CBF
:10F930000AB10F221A54704764C8FF1F014B185CAC
:10F94000704700BF64C8FF1F414B41F2300170B5E2
:10F950005A58404C404D42F000625A5041F23C022D
:10F9600003F58250995841F000619950016841F0C7
:10F9700002010160995841F00201995037490C2366
:10F980008B601023CB60364B00224A621A625A62A7
:10F990009A6244230B6004230B62B823A370314B9B
:10F9A00003F582506FF00206056041F24405012024
:10F9B000585341F24C055E5141F25005595141F204
:10F9C000540141F25E055A5241F258015A5041F237
:10F9D000480158500321595341F25605595341F2F9
:10F9E00046055A5341F25C055853A920E07003F5CF
:10F9F000835004F51A241034046041F264006FF05F
:10FA000005041A5241F26C001A5041F27002164875
:10FA1000985041F2740002221A5241F278001C50B0
:10FA200041F268001A5041F27E0048F203421A5235
:10FA300041F276001A5241F2660240F201109852E9
:10FA400041F27C024FF408709852D97670BD00BF25
:10FA500000700440001002404CC0FF1F00B00B407B
:10FA600000B00440008000408CC8FF1F09282BD83C
:10FA7000DFE800F0050A0D1014172A2A1A25134B87
:10FA80001888C0F30B107047104B5888F9E70F4BDC
:10FA90009888F6E70D4B188880B270470B4B588852
:10FAA000FAE70A4B9888F7E7084B588883B24FF477
:10FAB000987058434FF6FF7390FBF3F07047034B79
:10FAC000988883B23420F4E7002070478CC8FF1F69
:10FAD00030B52E4D41F23C042B5943F010032B510D
:10FAE0002B4B4FF400749C646FF4F875DC64A3F541
:10FAF0001833A4F13E542C441C604FF400545C6055
:10FB0000244C1C601C68E401FCD50138072834D85B
:10FB1000DFE800F0312F2D2B293327041E485860D1
:10FB20001E4B002058631E4818601E484FF080642A
:10FB300000EA8145C3F88040C3F88450FAB100EA76
:10FB40008240C3F89040C3F894004FF08460C3F83B
:10FB5000A000C3F8A410AAB1C3F8B000C3F8B42041
:10FB600030BD1148DBE71148D9E71148D7E7114804
:10FB7000D5E71148D3E71148D1E71148CFE7C3F8DB
:10FB80009020E2E7C3F8B02030BD00BF0070044011
:10FB900000A004400F0080508320FC010040024080
:10FBA0000F0080000000FC1F8720FE028720FE0B54
:10FBB0008720FE0E8720FE1D8720FE4A8720FE95A7
:10FBC0008720FE05384AD2F88030C3F30363022B46
:10FBD0005FD0D2F89030C3F30363022B5BD0D2F82E
:10FBE000A030C3F30363022B06D0D2F8B030C3F3C6
:10FBF0000363022B56D103231B0103F1402202F5BC
:10FC00000032D2F88010C1F303410170D2F88010A5
:10FC100011F4801118BF01218170D2F8801011F405
:10FC2000001118BF012141704178B1BBD2F8841096
:10FC3000C1F38A4103F1402303F500334160D3F857
:10FC40008810090E0172D3F88810090C4172D3F89C
:10FC50008810090A8172D3F88810C172D3F88C1009
:10FC6000090E0173D3F88C10090C4173D3F88C1072
:10FC7000090A8173D3F88C30C373D2F880309B02A9
:10FC80004CBF4FF084634FF08063C2F88030012096
:10FC900070470023B0E70123AEE7D2F8841021F0CB
:10FCA0006041C7E70020704700400240184AD2F880
:10FCB0007031C3F303630C2B10B527D0447843682D
:10FCC00004B3C3F31103C2F874318368104A1BBA3A
:10FCD000C2F87831C3681BBAC2F87C318378002C33
:10FCE00014BF4FF042624FF040620BB142F48012F9
:10FCF00003781B0403F470231343054A0120C2F860
:10FD0000703110BD034901EA8343DCE7002010BDD8
:10FD1000004002400000FC1F0B4B4FF00062C3F894
:10FD200070214FF48022C3F87421084AC3F8782167
:10FD30006FF48471A2F166320A44C3F87C21044A4C
:10FD4000C3F87021704700BF00400240785634125B
:10FD50000000080C10F0040F0A4B10D04FF4804242
:10FD6000C3F8A020C2064CBF074A084A9A6310F0A5
:10FD70000800074B1ABF01221A70187070474FF421
:10FD80008072F3E70090044000010A0000010900BE
:10FD900098D4FF1F38B50446F8F790FD0C49E517D5
:10FDA000C1E90045D1E900452B0243EA1463220270
:10FDB000C1E90023074A00231360074A1360074A7A
:10FDC000D3645360D364BDE83840F8F773BD00BF17
:10FDD00060CDFF1F1CCDFF1F18CEFF1F00900340FA
:10FDE0000D490E4A4FF4804330B5C1F8A0300C4B9A
:10FDF00000240025C3E9004500231360094A13606D
:10FE0000094AD3645360D364084B1B7813B94FF489
:10FE100080738B6330BD00BF0090044018CEFF1F7D
:10FE200060CDFF1F1CCDFF1F0090034098D4FF1F23
:10FE300010B9024B09011960704700BF58CDFF1F70
:10FE400008B9084686E7704730B9044BD3E9002368
:10FE5000100A40EA036070470020704760CDFF1F22
:10FE600008B9084696E770472A4941F23C0210B5A6
:10FE70008B58294C43F000738B50284B5A6D42F03D
:10FE800004025A651A6822F018021A605A6D22F0AC
:10FE900001025A65D3F8842042F0C002C3F88420DE
:10FEA00000214FF6FF72D96459609A60D3F8802020
:10FEB00042F00102C3F88020D3F8802042F02002F3
:10FEC000C3F88020D3F8802042F01002C3F88020CD
:10FED0005A6D42F001025A651A6842F008021A602F
:10FEE0004FF4E063236363630D4B0E4A18694309C3
:10FEF0001B0100F01F001360FFF72CFF0846FFF7FF
:10FF000049FF4FF48043C4F8A0305720BDE81040AB
:10FF100000F022B8007004400090044000900340BC
:10FF2000B8CDFF1F58CDFF1FFEE74FF0E023084A72
:10FF3000C3F8082D074A4CF22053D3814DF62813FD
:10FF4000D381138823F001031B041B0C138070471B
:10FF50000080000000200540802800F01F014FF0C5
:10FF600001030F4A04DD8B40C2F88C31D360704727
:10FF7000402804DD8B40C2F8883193607047202808
:10FF800004DD8B40C2F8843153607047404200F07A
:10FF90001F0058BF41428B40C2F880311360704748
:10FFA00000E100E0802800F01F024FF001030D493E
:10FFB00003DD9340C1F88C307047402803DD934047
:10FFC000C1F888307047202803DD9340C1F88430A1
:10FFD0007047404200F01F0058BF42429340C1F8B2
:10FFE0008030704700E100E0074B1A78D2B2012A56
:10FFF00002D1222903D15A7001225A707047212957
:020000021000EC
:10000000FAD10022F7E700BF92C8FF1F70B515466E
:1000100011B91B4B197070BD022903D1184B012275
:100020001A7070BD04291AD1154B5B78012B25D1AC
:100030009488402C28BF402400235E1CDBB2A342DE
:1000400007D300231A4602211846BDE8704000F08D
:1000500047BF2A68D05C00F0C3F83346EDE70329B8
:1000600006D1074A5378012B08D100239370E9E7A2
:10007000052901BF024B00221A705A7070BD00BFE3
:1000800092C8FF1F10B50446204600F0C1F80028B2
:10009000FAD110BD704738B50A4C012502460B460F
:1000A00000202946A57000F0F5FA224618B1002379
:1000B000A370122038BD937803F0FF00002BFAD113
:1000C00038BD00BF92C8FF1FF8B506460F4600F0C6
:1000D000F4FC0E4B1A78012A16D15B78012B13D150
:1000E00000F000F988B10025ECB2A74205D82146FE
:1000F0003046BDE8F840FFF7CEBF301900F0D6F823
:1001000001350028F0D0F2E70C20F8BD92C8FF1F9F
:1001100008B540210248FFF7D7FF00F095F808BD69
:1001200095C8FF1F38B5054600F0A8F80B2804460F
:1001300009D140210548FFF7C7FF28B92846BDE887
:10014000384000F09BB80024204638BDD5C8FF1FBA
:1001500070B50C46461E00250CB9284670BD16F831
:10016000010FFFF7DFFF013C002818BF0B25A4B2E9
:10017000F2E738B5451E002415F8010F08B92046EE
:1001800038BDFFF7CFFF002818BF0B24F4E707B5F1
:100190000123002200930649064B104600F020FA86
:1001A000002814BF1B20002003B05DF804FB00BF33
:1001B0000D000100E9FF000038B50C46054600F0CF
:1001C00097F8A0420AD32C440020A54207D000B1E2
:1001D00038BD15F8010B00F051F8F6E70B2038BDDB
:1001E00010B50A4A117840290ED05378D41801333B
:1001F000DBB2402BA07001F101014FF00000117043
:1002000014BF5370507010BD0B2010BD15C9FF1FD7
:1002100010B50C4A117891B192F84230D4180133DC
:10022000DBB2A4780470402B4FF0000001F1FF31E5
:10023000117014BF82F8423082F8420010BD0A20CB
:1002400010BD00BF15C9FF1F014B1878704700BFD4
:1002500015C9FF1F024B1878C0F14000C0B27047AB
:1002600015C9FF1F034B00225A7083F842201A70F1
:10027000704700BF15C9FF1FFFF7F4BF10B50A4A4A
:10028000117840290ED05378D4180133DBB2402BBB
:10029000A07001F101014FF00000117014BF537004
:1002A000507010BD0B2010BD58C9FF1F10B50C4A6F
:1002B000117891B192F84230D4180133DBB2A478AE
:1002C0000470402B4FF0000001F1FF31117014BF9A
:1002D00082F8423082F8420010BD0A2010BD00BFF3
:1002E00058C9FF1F014B1878704700BF58C9FF1F3E
:1002F000024B1878C0F14000C0B2704758C9FF1FC8
:10030000034B00225A7083F842201A70704700BFD6
:1003100058C9FF1FFFF7F4BF70B50546007801F01C
:1003200093F902780023D9B2914207D25C1C03EB07
:10033000830303445E786B789E4227D1174C2B7A57
:10034000342202FB0142D67813B334234B43E21824
:10035000907886420CD000F0030204330C2010FB8E
:1003600002302118205C0B894A68497800F090FB24
:10037000D4F89C3083B12A46287812F8081F002947
:100380000CBF03210521BDE8704018472346CAE78A
:10039000937801339370D8E770BD00BF9CC9FF1FED
:1003A0002DE9F04F85B00D4690468DF80F0001F015
:1003B0004BF9022D064647D1077800235C1CDBB2BF
:1003C000BB4210DB4FF00009DFF8B0B0CA465FFA5D
:1003D00089F4A74212DC284BD3F89C30002B45D17E
:1003E00005B0BDE8F08F03EB830333440DF10F003C
:1003F000DA78597801F0E2F92346DFE704EB840468
:100400003444E378A2886178CDF804A0A078009005
:100410000DF10F0001F0B0F9A378032B05D15A4676
:1004200061789DF80F0001F031FA6178E37841F0CE
:10043000100141EAC3110022C9B20DF10F0001F011
:10044000EDF909F10109C2E7002DC4D10A49037889
:10045000342000FB03138A1C3633294634329A4277
:10046000B9D002F8341C02F8331CF7E7424629469B
:100470009DF80F009847B3E79CC9FF1F19030100BF
:10048000F0B40C7804F06004202C1D4632D14C7876
:10049000042C1DD00AD8012C04D003D3022C20D068
:1004A000032C12D000202880F0BC7047212C1BD0D8
:1004B00004D8202CF6D1F0BC00F040B9222C16D084
:1004C000232CEFD1F0BC00F049B9F0BC00F049B9E1
:1004D00002241C801468002525701468671C1760AE
:1004E0006570F0BC00F056B9F0BC00F01FB9F0BC6C
:1004F00000F076B9402C06D1044CD4F8A04014B1D9
:10050000A446F0BC6047CD20CEE700BF9CC9FF1FCA
:1005100073B50446007801F097F863680093A27AF7
:10052000637A43EA0223ADF8043002780023D9B29B
:10053000914207D25D1C03EB830303445E7863782A
:100540009E4225D1174D237A342202FB0152D678E0
:1005500003B334234B43EA18907886420CD000F062
:10056000030204330C2010FB02302918285C0B898D
:100570004A68497800F08CFAD5F89C3033B1227A79
:1005800020785AB104F108020521984702B070BDE5
:100590002B46CCE7937801339370DAE76A46032160
:1005A000F3E700BF9CC9FF1F07B543680093437A78
:1005B000817A43EA0123ADF80430084BD3F89C302C
:1005C00002462BB1017A007829B1083205219847FB
:1005D00003B05DF804FB6A460421F8E79CC9FF1FDD
:1005E0002DE9F84305460F461646984601F02CF8CB
:1005F00002789DF8203001328146D2B2002128468F
:1006000001F09EF80446E8B9164A1749284600F05A
:1006100086F999F80000154B342200FB022209F1FB
:1006200001011A4499463433934201F105010CD17A
:100630004146284600F074F8044618B9C9F89C7081
:10064000C9F8A0602046BDE8F88311F8050C03F84E
:10065000340C11F8040C03F8330C03F8324C03F893
:10066000314CE0E781040100A10301009CC9FF1F98
:1006700008B5074B0022C3F89C20C3F8A02000F067
:10068000A1F918B9BDE8084001F06EB808BD00BF77
:100690009CC9FF1F2DE9F041984605460E461746B6
:1006A00000F0D2FF04780023D9B2A14207D201336F
:1006B00003EB8302024412F8042CB242F4D1174C2B
:1006C00034234B43E218D07892F802E0A0EB0E01FD
:1006D000C9B2042902D1C120BDE8F08100F00301B4
:1006E0000130C0B24FF00C0C0CFB0133D070A0EB0A
:1006F0000E001C44C0B2012825716671A760A4F8E1
:100700000C8007D143463A4631462846BDE8F041C1
:1007100000F0BEB90020BDE8F08100BF9CC9FF1FFA
:10072000014B00201960704740CAFF1F024B097936
:10073000197100F08DBF00BF40CAFF1F13B5002420
:1007400002AA1C80044B42F8041D0979197100F0BB
:100750008DFF02B010BD00BF40CAFF1F00201880EF
:10076000704730B40C460221198021796488084D05
:10077000012C297102D130BC00F08EBF022C02D1B5
:1007800030BC00F095BF0020188030BC704700BF1F
:1007900040CAFF1F30B40C460221198021796488B9
:1007A000074D012C297102D130BC00F08DBF022C05
:1007B00002D130BC00F09ABF0020188030BC7047D6
:1007C00040CAFF1F044B054A19795B7911711372F6
:1007D00003210A23FFF75EBF40CAFF1F4FC0FF1F60
:1007E000F8B500271F808B780B4CA371C3F340032F
:1007F0005A0063F3000206466271FFF7E3FF2568C3
:1008000045B1A37913F002021ABF3A4622212121F1
:100810003046A8470020F8BD40CAFF1F034B00F137
:1008200008021B6800780521184700BF48CAFF1F4F
:1008300070B5094D04462A1D012100F0D7FF802222
:100840000121204600F0EAFF2B68207800220A21CF
:10085000BDE87040184700BF48CAFF1F37B50121E7
:100860000DF10702044600F0C1FF9DF80730074D67
:10087000802B04D12A790121204600F0CFFF2B687C
:10088000207800220B21984703B030BD48CAFF1FD3
:10089000436805215A7800F0C1BF73B501220024D6
:1008A00005460126002100F089FF334621468DE8E8
:1008B00050001022284600F05FFF224621462846BD
:1008C00000F07CFF234621468DE850001022284688
:1008D00000F052FF31460222284600F09FFF3246C8
:1008E0000621284600F09AFF22469021284600F073
:1008F00095FF044B28781B682246214602B0BDE8CC
:100900007040184748CAFF1F42783AB9C178C901F8
:1009100041F0100101F0900100F080BF704773B505
:100920000C468DF8070001F00DFA1F4D2C600446AF
:10093000002836D11D4A9DF80700102100F0A6FFBF
:100940001B4A044612219DF8070000F09FFF194A38
:10095000044314219DF8070000F098FFE4B204431B
:10096000154A9DF80700132100F090FFE4B20443FC
:10097000124A9DF80700172100F088FF02AEE4B28A
:1009800004430F4A16F8010D162100F07FFFE4B270
:10099000044303220121304600F040FF0323E4B268
:1009A0002B71204602B070BD48CAFF1F9B08010092
:1009B00091080100310801005D08010009090100EA
:1009C0001D08010037B502AD174B05F8010D0022D7
:1009D000102128461A6000F05BFF122104462846C9
:1009E00000F056FF14210443284600F051FFE4B202
:1009F00004431321284600F04BFFE4B204431721BF
:100A0000284600F045FFE4B204431621284600F0D2
:100A10003FFFE4B2204310F0FF0003D19DF8070030
:100A200001F09CF903B030BD48CAFF1F1FB501217A
:100A30008DF807000DF10E020DF1070000F0D6FE53
:100A40000DF10F0206210DF1070000F0CFFE9DF819
:100A50000E30802B18D19DF80F309B0714D59DF8D0
:100A6000070000F0EFFD012804460DD172B60DF12C
:100A7000070000F029FB002221460DF107008DF848
:100A80000E2000F0CBFE62B69DF80E0004B010BD43
:100A900073B50C4615461E468DF80700FFF7C6FFD6
:100AA000802808D033462A4621460DF1070000F081
:100AB000A7FA02B070BD0020FBE77047062812D8E5
:100AC00080000129C0B201D10230C0B2074AC0F390
:100AD0004703122101FB03231A884FF6FF739A4242
:100AE00008BFFF207047FF20704700BF50CAFF1F9C
:100AF0002DE9F041314C324D324E4FF0000884F870
:100B000000814FF4107285F840020F462846FF21FD
:100B100002F072F94FF4806241463046C5F84462F3
:100B200002F06AF994F80C3143F0800384F80C3138
:100B300094F80C311B06FBD4234BFF221A7094F857
:100B40000C3143F0400384F80C31204B196897B303
:100B500041F000411960194B310AC6F3074201F018
:100B6000FE0183F89C1083F8B020320E83F8B42085
:100B7000174AC5F84822102283F80821012283F879
:100B80009420BF2283F8802093F8002102F07F0296
:100B900083F8002193F8842042F0010283F8842036
:100BA00093F8842042F0100283F8842084221A777C
:100BB0000020BDE8F08121F00041CBE70020074094
:100BC00050CAFF1F00D6FF1F59C0FF1F007004400E
:100BD00000D8FF1F0D4B93F80C2102F0BF0283F8E1
:100BE0000C21BF2283F8802093F8842002F0FE02BB
:100BF00083F8842093F8942002F0FE0283F8942076
:100C00001A7F02F07B021A7700207047002007400D
:100C1000F7B5082304248DE81800B1F803300D78E7
:100C20008878B3F5007F81BF0023CB7002230B715E
:100C3000062D71D8AB00DCB2012804BF0234E4B247
:100C40004FEA540E354C122707FB0E474FF6FF763E
:100C5000B7F800C0B4455FD14E78032E5CD80128A8
:100C60005AD897F80FC0BCF1FF0F04BF4FF0000C2B
:100C700087F80FC0B1F803C0122101FB0EFE04EB90
:100C80000E0743EA4003BA73FA7B7E7402F0010256
:100C900013435BB2D4F84822C7F80220D9B2F973E3
:100CA0003874D4F8447224F80EC01BB207EBC30E9C
:100CB00081F00101CEF80420AEF802C04FF0080E1A
:100CC00007F833E007EBC10ECEF80420AEF802C0FF
:100CD00012FA8CF24FF0480E07F831E0C4F84822BF
:100CE00028B917F8332062F07F0207F8332002AAF0
:100CF00002EB80002DB20A4950F8082C11F825307B
:100D0000012E0CBF164642F001063343DBB201F858
:100D10002530002003B0F0BD9520FBE750CAFF1F2F
:100D2000C0200740084610B51146FFF7C7FEFF2850
:100D30001DD0104B1221C0F3470001FB0030D3F847
:100D40004422C37B1CB283F0010312F8341001F07B
:100D50007F0102F8341012F8331001F07F0102F81D
:100D600033104FF0FF338372C372002010BDC420D4
:100D700010BD00BF50CAFF1F73B50C468DF80700A9
:100D8000114620461646FFF799FEFF28054620D05B
:100D9000214632460DF10700FFF7C4FFC5F34703B4
:100DA00012210D4D59436B18D5F848221888121A94
:100DB000C5F8482224B2094A002002F824004FF066
:100DC000FF326A549A705A70DA701A715A7102B00E
:100DD00070BD9620FBE700BF50CAFF1FC020074030
:100DE0002DE9F0410E468046114630461746FFF782
:100DF00065FE0C4DC0F34700122303FB0050C47B7B
:100E0000FF2C0DD03A4631464046FFF78BFF24B207
:100E1000D5F8442212F8343063F07B0302F8343002
:100E2000BDE8F08150CAFF1F10B5084600211446E6
:100E3000FFF744FE084AC0F34700122101FB0020DF
:100E4000D2F84432C27B03EBC2035A6813682360B2
:100E50005368636010BD00BF50CAFF1F10B50C4639
:100E600020461146FFF72AFEFF281AD024B2104B65
:100E700013F82430DBB213F00C0F12D09B0712D4FE
:100E80000C4BD3F8443213F83020D2090DD180F046
:100E90000100C0B213F83030DB0914BF032000207A
:100EA00010BD052010BD012010BD032010BD00BFE6
:100EB000C020074050CAFF1F08B5FFF7FFFD074AD3
:100EC0001223C0F3470003FB0020C37BFF2B1EBF90
:100ED000D2F84422002102F8331008BD50CAFF1F87
:100EE0002DE9F0410846002190461F46FFF7E6FD38
:100EF0002249C0F34700122404FB0014E57BFF2DB8
:100F000039D022884FF6FF7093B2834233D0D1F8A4
:100F1000441285F0010011F9300000282BDB2EB2BD
:100F200087B901EBC60338465A80D4F802205A60CC
:100F300011F8352002F0400262F0770201F8362005
:100F4000BDE8F08101EBC602BB424FF0000028BFB4
:100F50003B466781C4F80680207360735380C2F8F3
:100F6000048011F8353003F0400363F0770301F893
:100F70003630BDE8F0819420BDE8F08150CAFF1FF3
:100F80002DE9F0410C460646114620461546FFF76E
:100F900095FD194BC0F34700122202FB003090F878
:100FA0000FE0BEF1FF0F24D027B2144A6CB1407C91
:100FB000012D0CBF14211821012818BF41F0010197
:100FC00012F82700014302F8271012F827106FF3D8
:100FD000410102F82710D3F84432002203F83E20E2
:100FE0003DB92B462A4621463046BDE8F041FFF781
:100FF00077BFBDE8F08100BF50CAFF1FC020074087
:101000002DE9F0410C462046012117469846FFF78E
:1010100055FDFF2836D01C4BC0F34700122202FBBF
:101020000030D3F8446290F80FE016F93E30002B00
:1010300028DB23B2154A12F8235015F0020521D1FE
:101040000188C0F806701FFA88F242818A42D8BF30
:1010500011460FFA8EF206EBC203057345735980F1
:101060005F602CB9C82306F832302046BDE8F08115
:1010700016F83E3003F0400363F0770306F8323091
:101080002C46F2E79324F0E750CAFF1FC020074028
:10109000034B044883F898100122114600F0BEBBB0
:1010A0000020074090CCFF1F054B0648002283F824
:1010B0009420802283F80C210121FF2200F0AEBB96
:1010C0000020074090CCFF1F38B51A4C94F800213F
:1010D00002F07F0284F8002194F80C2102F0DF0274
:1010E00084F80C2194F8802042F0200284F88020BB
:1010F00094F8842002F0DF0284F8842094F894208D
:1011000002F0DF0284F8942094F8942042F0040264
:1011100084F8942044F62065013DADB200F0BCFE99
:10112000002DF9D194F8943003F0FB0384F8943047
:1011300038BD00BF002007402DE9F04FD84DD94CF5
:1011400095F8807095F8843095F8906087B0FF220C
:101150001F4094F840328DF809208DF80C308DF83E
:101160000D20002301210DF1090204F510708DF806
:101170000E3004938DF815308DF816308DF80F3041
:101180008DF8143000F032FB95F80C31D907F6B227
:101190000FD59DF80930802B0BD195F8003103F065
:1011A0007F0385F8003195F80C3103F0DF0385F8F3
:1011B0000C317A0711D5BA4B042093F8A41093F898
:1011C000A02083F8800006AB42EA012223F80E2D0E
:1011D00003A91220049300F06DFBFB074BD5B04D23
:1011E000B0480123BF2685F8803085F8886095F8DF
:1011F0009430002743F0020385F894304FF41072C6
:1012000085F89870FF2185F8007101F0F5FD4FF425
:1012100080623946D4F8440201F0EEFDD4F844323D
:1012200003F50073C4F848329F4BFF221A7095F8FB
:10123000943003F0FD0385F8943095F80C3143F0B9
:10124000400385F80C319F2385F88C6085F8843045
:1012500095F8943003F0DF0385F8943003A910204B
:1012600000F028FB95F8943003F0DF0385F8943004
:1012700007B0BDE8F08F3D0740F19380884B08220E
:1012800083F880203309C6F3C000062B8DF80D309B
:101290008DF80F0000F2F480C6F3800202EB8302A7
:1012A00008B10232D2B2D4F8446206EBC201C2F3F2
:1012B0004705D1F804E04988ADF81510122101FB6B
:1012C0000541CDF810E091F80FC08CF0010C81F8C9
:1012D0000FC016F8321082F0010A5FFA8AFAC1F3E1
:1012E00080110FFA8AF881F00101890106EBC80923
:1012F00006F83810002800F0D980DFF8ACB19BB9AF
:101300009BF8002082B9FF2219468BF8002003A821
:101310001A460193FFF706FD019B06F838301A467E
:10132000194603A8FFF7DCFD9BF80030012B04D021
:101330009DF80D30002B00F0AD80122101FB05411E
:10134000BDF815008B894A8903449BB293428B8177
:1013500009D3B1F800E0C0B2864540F09380897BA4
:10136000012940F08F80122101FB0544D4F80610BA
:1013700020881944D31A8342D8BF98B2A9F8020032
:10138000C9F8041016F83A3003F0400363F077030D
:1013900006F83830424A92F8943003F0DF0382F8BE
:1013A0009430B80717D53E4C022384F8803094F867
:1013B000883094F88C2003A9134016208DF814303F
:1013C00000F078FABF2384F8883094F8943003F062
:1013D000DF0384F89430F9061CD5314C202384F8BF
:1013E0008030102384F8803003A9142000F062FAC2
:1013F00094F80C3143F0200384F80C3194F8003158
:1014000043F0800384F8003194F8843043F02003E3
:1014100084F88430BA060DD5214C202384F880301E
:1014200003A9132000F046FA94F8843003F0DF0398
:1014300084F884303B067FF51BAF0DF10A02FF23D1
:10144000102103A88DF80D3000F0D0F99DF80A3076
:10145000134C012B04BF8DF80F3000224FF0800396
:1014600008BF8DF80D2003A984F88030172000F004
:1014700021FA94F8943003F0DF0384F89430F7E60F
:10148000FF2210E7122202FB0544D4F80620049242
:10149000ADF8153003A99DF80D0000F00BFA79E7BF
:1014A0000020074050CAFF1F59C0FF1F6BB916F834
:1014B00032202F4902F03C02342A35D101238DF825
:1014C0000E309EF80030DB090B70122101FB054144
:1014D0004FF6FF734A899A42DCD0BDF815E08B893C
:1014E00073449BB28B8109888E4501D19A420CD8F6
:1014F0008AB3B2FBF1F001FB102080B258BB12207E
:1015000000FB0540807B012825D1D21A8A42D8BF32
:1015100091B2122202FB0544C9B9D4F80230C9F8CD
:101520000430A9F802102DE70A78012ACDD1FF2056
:101530000870194603A80193FFF7F4FB019B06F816
:1015400038301A46194603A8FFF7CAFCBDE7D4F89D
:1015500006201344E3E7122202FB0544D4F80620D8
:10156000ADF815304FF0FF330492A372E37291E7A8
:1015700059C0FF1F13460A46194601F03DBC00BF83
:1015800030B50329039C04981DD12BB9164A22605B
:1015900004220280002030BD40F209418B420FD16D
:1015A000022A4FF000030CD810490C2505FB031349
:1015B000D9681B6951F8221021609B5C0380E9E720
:1015C00001230122F0E7072901D9CD2030BD074BC7
:1015D00003EB8102126A2260002AF6D003EB41037A
:1015E000B3F84030EAE700BF5AC0FF1F34300100B3
:1015F00001299FBF034B5B5C1370002088BFCD2087
:10160000704700BF9CCCFF1F01299DBF024B0020EB
:101610005A54CD20704700BF9CCCFF1F19B14B1E00
:1016200058425841704701207047054B1A788A424A
:1016300004D05878431A58425841704701207047E7
:101640009CCCFF1F00207047004870478430010089
:1016500001299FBF044BC1EBC101C918002094BFF1
:101660001160CD20704700BF5EC0FF1F012930B55B
:101670000ED8084DC1EBC10108231068C45CC8181E
:10168000284401330F2B00F8084CF6D1002030BD60
:10169000CD2030BD5EC0FF1F01299FBF034B03EB70
:1016A00041010020116088BFCD2070479ECCFF1FF4
:1016B00001299FBF034B03EB41010020116088BF4C
:1016C000CD207047A2CCFF1F01290AD813681878D3
:1016D000054B03EB4101887013685B78CB700020E9
:1016E0007047CD20704700BF9CCCFF1F01290AD84E
:1016F00013681878054B03EB4101887113685B7818
:10170000CB7100207047CD20704700BF9CCCFF1FDD
:10171000084B5A7803F8022BFF210022D1540132E2
:10172000072AFBD1044A0023052199540133072BD2
:10173000FBD17047A6CCFF1FAFCCFF1F00BF704787
:10174000013AD2B2062A10B51C4608D8054B5A7089
:10175000FFF7DEFF2146BDE81040FFF7C9B9992029
:1017600010BD00BFA6CCFF1F024B00225A70FFF72E
:1017700031BA00BFA6CCFF1F37B50F4C257805B98D
:10178000C1B98DF802308DF800109DF81830ADF811
:10179000032069469DF81C2000788DF80130FFF782
:1017A00037FA9DF800301BB110B92378013B237044
:1017B00003B030BD9520FBE7A6CCFF1F38B50A4B20
:1017C0000D461C7859788C421C4600D14DB92946EB
:1017D0000078FFF7D1FA2DB120B9237801332370B7
:1017E00038BD962038BD00BFA6CCFF1F4B1E062B70
:1017F00005D8094B19444B78137000207047CB066D
:1018000007D501F00F01062903D8034B19444B7A81
:10181000F2E78220704700BFA6CCFF1F4B1E062BAD
:101820002DE9F0418046174605D8174B19444A70F8
:101830000020BDE8F081CB0622D501F00F05062D72
:101840001ED8012A4FEAD1140F4E06D1224629464E
:10185000FFF7C6FA35446F72EAE7002AFAD1731926
:101860005B7A012BF6D122462946FFF789FB002D32
:10187000F0D184F0010229464046FFF781FBE9E7F9
:101880008220BDE8F08100BFA6CCFF1F002070477A
:10189000062903D9A1F11003072B07D8044B53F8ED
:1018A0002130002B0CBFC42000207047C42070479B
:1018B000AC300100102810B50C4601D1FFF728FF0D
:1018C000034B53F820300BB120469847002010BD41
:1018D000AC3001001FB5144602228DF807001A80B3
:1018E00005210DF10F020DF10700FFF77FFF034BFC
:1018F0009DF80F201A80236004B010BDB8CCFF1FE4
:101900001FB5144601228DF807001A8004210DF13D
:101910000F020DF10700FFF769FF044B9DF80F2040
:101920001A800020236004B010BD00BFB8CCFF1F98
:10193000F0B5002685B01E8049888DF80700ADF807
:101940000E10FFF76BFE18B3BDF80E20114F04AC5C
:10195000B2FA82F2520901210DF10700FFF75EFF92
:1019600034F8022D0421D2B20DF10700FFF756FF23
:101970007B682246012105469DF8070098477B6851
:101980009DF80700324602219847284605B0F0BD71
:101990000425FAE7B8CCFF1F73B502AC002504F8A4
:1019A000010D0E461D80042201212046FFF736FF5F
:1019B0007288024B28461A7202B070BDB8CCFF1F65
:1019C00013B54C8889888DE80C000B46E2B2210AD9
:1019D000FFF7D6FD02B010BD2DE9F04186B01746E5
:1019E0001E4606AA00238846059303238DF80F00A0
:1019F00002F8083D01210DF10F00FFF7F7FE98F8FE
:101A00000050274C15F0030528D10DF111020621D5
:101A10000DF10F00FFF7EAFE9DF811309DF80F0061
:101A200003F0030323800DF11203019305AB009330
:101A30002A462B460221FFF7A3FD059BDB7913F015
:101A4000400F238814BF43F0010323F001032380D8
:101A5000022333803C6006B0BDE8F081012D08D13F
:101A60009DF81030012B02D198F80430ABB9002357
:101A7000EDE7022DEED198F8041041F010010DF1C0
:101A80001202C9B20DF10F00FFF7B0FE9DF812303F
:101A900003F0010323803580DCE7CD20DAE700BFC7
:101AA000B8CCFF1F7FB500221A800B784E788DF8D6
:101AB000070013F003030D46C6F3400634D1FEB110
:101AC0004B88013B9BB2012B52D80DF10F0206212E
:101AD0000DF10700FFF78AFE044670B9AB780122CA
:101AE0009A409DF80F301A43D2B206210DF107003B
:101AF0008DF80F20FFF792FE0446204604B070BD1B
:101B00004E88012E34D10DF10F0206210DF1070090
:101B1000FFF76CFE04460028EFD1AA7896409DF8A6
:101B20000F2022EA0602E0E7022B21D109798DF885
:101B30000F10324641F010010DF10700FFF76EFE65
:101B40006B78002E14BF07210821012B044607D112
:101B50009DF80F00C10900F00F00FFF7ADF9082153
:101B6000044B9DF807005B680DF10F029847C4E72E
:101B7000CD24C2E7B8CCFF1F10B500241C800B7821
:101B800003F00303012B05D18A780979FFF73CFDA7
:101B9000204610BD042010BD38B515460A7802F065
:101BA0000302012A07D1054C1A8009792246FFF762
:101BB0001FFD2C6038BD042038BD00BFB8CCFF1F0E
:101BC00013B5CD298DF8070007D1012290210DF121
:101BD0000700FFF723FE02B010BD0D491C88088ADC
:101BE0001268844288BF18800C461B889DF8070045
:101BF0000021FEF74DFF94F90A30002BEBDA0023A9
:101C00001A4619460DF10700FFF76AF9E3E700BF2E
:101C1000B8CCFF1F73B5054600266A4601218DF832
:101C200000600196FFF7E2FDAA78434C012A52D1E9
:101C300068680368C4F80A304368A07AC4F80E30B4
:101C400004F10A0110F0600F1ED1E27A3B4B53F809
:101C50002240002C3DD09DF80000022839D802EB2C
:101C600042021344034493F83430012B31D10DF177
:101C7000020301AA2878A0470DF1020301AA014638
:101C80002878FFF79DFF13E0238AADF80230202B60
:101C900017D87BB102060DD40A68C4F812204A682E
:101CA000C4F81620314604F11A022846FFF718F945
:101CB00002B070BDE46B64B10DF1020301AA2049CA
:101CC000D8E702A82B7800F8073D9021FFF7A6FD82
:101CD000EEE7CD20D0E79DF80030042B10D12B7813
:101CE000217A02AD05F8063D2846FFF7D1F9012219
:101CF00011462846FFF792FD227A03212846E5E7A0
:101D000094F90A30002BD3DBEB78002BD0D1E66BB3
:101D100086B1B5F8093028780833ADF8023004F1FF
:101D200012010DF1020301AAB04701460DF10203B1
:101D300001AAA5E7CD21F9E7B8CCFF1F0C310100BE
:101D4000C2CCFF1F034B5960DA630021024AFFF740
:101D50009DBD00BFB8CCFF1F151C010007B502AB2D
:101D6000054A03F8010D002118465160D163FFF7C1
:101D70008FFD03B05DF804FBB8CCFF1F0020704757
:101D8000354B41F248015A5822F00D0242F005024B
:101D90005A5041F204015A5842F480225A5041F2FA
:101DA00034015A5842F480225A5003F52C336021F2
:101DB00093F8942042F0020283F89420C02283F822
:101DC0000021FF221A7483F8802083F8882083F88A
:101DD0008420002283F88C2083F80C111F491A7587
:101DE000080A00F0FE0083F8982083F8C02083F8EA
:101DF000C42083F8C82083F8CC2083F8D02083F84F
:101E0000D42083F8D82083F8DC2083F8E02083F8FE
:101E1000E42083F8E82083F8EC2083F8F02083F8AE
:101E2000F42083F8F82083F8FC2083F89C00C1F3A9
:101E30000740090E83F8B00083F8B41083F8AC2093
:101E40001A7783F8082193F8942002F0D40242F024
:101E5000010283F8942070470070044000D6FF1FF1
:101E6000024B4FF400729A60704700BF00E100E03F
:101E7000034B4FF40072C3F888219A60704700BF8B
:101E800000E100E008B5FEF782F910B9FFF7F0FFB6
:101E900008BD1B2008BD00BF034B4AF202629A81B5
:101EA0004BF280429A8170470020054081F000414A
:101EB00002E000BF83F0004330B54FEA41044FEA2F
:101EC000430594EA050F08BF90EA020F1FBF54EACA
:101ED000000C55EA020C7FEA645C7FEA655C00F066
:101EE000E2804FEA5454D4EB5555B8BF6D420CDD37
:101EF0002C4480EA020281EA030382EA000083EABA
:101F0000010180EA020281EA0303362D88BF30BD59
:101F100011F0004F4FEA01314FF4801C4CEA1131AF
:101F200002D0404261EB410113F0004F4FEA03330E
:101F30004CEA133302D0524263EB430394EA050F99
:101F400000F0A780A4F10104D5F1200E0DDB02FA08
:101F50000EFC22FA05F2801841F1000103FA0EF29C
:101F6000801843FA05F359410EE0A5F120050EF162
:101F7000200E012A03FA0EFC28BF4CF0020C43FA93
:101F800005F3C01851EBE37101F0004507D54FF0A0
:101F9000000EDCF1000C7EEB00006EEB0101B1F5F0
:101FA000801F1BD3B1F5001F0CD349085FEA300036
:101FB0004FEA3C0C04F101044FEA445212F5800F41
:101FC00080F09A80BCF1004F08BF5FEA500C50F1DE
:101FD000000041EB045141EA050130BD5FEA4C0CC1
:101FE000404141EB010111F4801FA4F10104E9D14A
:101FF00091F0000F04BF01460020B1FA81F308BF41
:102000002033A3F10B03B3F120020CDA0C3208DD0C
:1020100002F1140CC2F10C0201FA0CF021FA02F1E7
:102020000CE002F11402D8BFC2F1200C01FA02F157
:1020300020FA0CFCDCBF41EA0C019040E41AA2BF7C
:1020400001EB0451294330BD6FEA04041F3C1CDA44
:102050000C340EDC04F11404C4F1200220FA04F064
:1020600001FA02F340EA030021FA04F345EA03010E
:1020700030BDC4F10C04C4F1200220FA02F001FAD0
:1020800004F340EA0300294630BD21FA04F0294652
:1020900030BD94F0000F83F4801306BF81F48011EB
:1020A0000134013D4EE77FEA645C18BF7FEA655C5E
:1020B00029D094EA050F08BF90EA020F05D054EA30
:1020C000000C04BF1946104630BD91EA030F1EBF35
:1020D0000021002030BD5FEA545C05D14000494139
:1020E00028BF41F0004130BD14F580043CBF01F52C
:1020F000801130BD01F0004545F0FE4141F4700112
:102100004FF0000030BD7FEA645C1ABF19461046EC
:102110007FEA655C1CBF0B46024650EA013406BFED
:1021200052EA033591EA030F41F4002130BD00BFAC
:1021300090F0000F04BF0021704730B54FF4806469
:1021400004F132044FF000054FF0000150E700BFEA
:1021500090F0000F04BF0021704730B54FF4806449
:1021600004F1320410F0004548BF40424FF0000136
:102170003EE700BF42004FEAE2014FEA31014FEA79
:1021800002701FBF12F07F4393F07F4F81F06051C8
:10219000704792F0000F14BF93F07F4F704730B537
:1021A0004FF4607401F0004521F0004120E700BFCA
:1021B00050EA010208BF704730B54FF000050AE051
:1021C00050EA010208BF704730B511F0004502D552
:1021D000404261EB41014FF4806404F132045FEA54
:1021E000915C3FF4DCAE4FF003025FEADC0C18BFF9
:1021F00003325FEADC0C18BF033202EBDC02C2F1EF
:10220000200300FA03FC20FA02F001FA03FE40EA80
:102210000E0021FA02F11444C1E600BF70B54FF080
:10222000FF0C4CF4E06C1CEA11541DBF1CEA135562
:1022300094EA0C0F95EA0C0F00F0DEF82C4481EACA
:10224000030621EA4C5123EA4C5350EA013518BFEA
:1022500052EA033541F4801143F4801338D0A0FBD7
:1022600002CE4FF00005E1FB02E506F00042E0FB84
:1022700003E54FF00006E1FB03569CF0000F18BF8A
:102280004EF0010EA4F1FF04B6F5007F64F5407432
:1022900004D25FEA4E0E6D4146EB060642EAC621C5
:1022A00041EA55514FEAC52040EA5E504FEACE2E32
:1022B000B4F1FD0C88BFBCF5E06F1ED8BEF1004F35
:1022C00008BF5FEA500E50F1000041EB045170BDB1
:1022D00006F0004646EA010140EA020081EA0301F5
:1022E000B4EB5C04C2BFD4EB0C0541EA045170BDF1
:1022F00041F480114FF0000E013C00F3AB8014F16B
:10230000360FDEBF002001F0004170BDC4F10004B3
:10231000203C35DA0C341BDC04F11404C4F1200534
:1023200000FA05F320FA04F001FA05F240EA02008F
:1023300001F0004221F0004110EBD37021FA04F6C5
:1023400042EB06015EEA430E08BF20EAD37070BD7F
:10235000C4F10C04C4F1200500FA04F320FA05F0DE
:1023600001FA04F240EA020001F0004110EBD370E0
:1023700041F100015EEA430E08BF20EAD37070BD50
:10238000C4F1200500FA05F24EEA020E20FA04F329
:1023900001FA05F243EA020321FA04F001F00041D8
:1023A00021FA04F220EA020000EBD3705EEA430E49
:1023B00008BF20EAD37070BD94F0000F0FD101F078
:1023C0000046400041EB010111F4801F08BF013CB1
:1023D000F7D041EA060195F0000F18BF704703F0EF
:1023E0000046520043EB030313F4801F08BF013D76
:1023F000F7D043EA0603704794EA0C0F0CEA135532
:1024000018BF95EA0C0F0CD050EA410618BF52EAEB
:102410004306D1D181EA030101F000414FF00000F1
:1024200070BD50EA410606BF1046194652EA4306FF
:1024300019D094EA0C0F02D150EA013613D195EA73
:102440000C0F05D152EA03361CBF104619460AD1BB
:1024500081EA030101F0004141F0FE4141F47001C5
:102460004FF0000070BD41F0FE4141F4780170BDB5
:1024700070B54FF0FF0C4CF4E06C1CEA11541DBF1A
:102480001CEA135594EA0C0F95EA0C0F00F0A7F81C
:10249000A4EB050481EA030E52EA03354FEA013149
:1024A00000F088804FEA03334FF0805545EA13135C
:1024B00043EA12634FEA022245EA111545EA106524
:1024C0004FEA00260EF000419D4208BF964244F1BB
:1024D000FD0404F5407402D25B084FEA3202B61ADA
:1024E00065EB03055B084FEA32024FF480104FF4AE
:1024F000002CB6EB020E75EB030E22BFB61A754622
:1025000040EA0C005B084FEA3202B6EB020E75EBB4
:10251000030E22BFB61A754640EA5C005B084FEA1C
:102520003202B6EB020E75EB030E22BFB61A7546E9
:1025300040EA9C005B084FEA3202B6EB020E75EBF4
:10254000030E22BFB61A754640EADC0055EA060EB5
:1025500018D04FEA051545EA16754FEA06164FEAF8
:10256000C30343EA52734FEAC2025FEA1C1CC0D1A4
:1025700011F4801F0BD141EA00014FF000004FF031
:10258000004CB6E711F4801F04BF01430020B4F1F2
:10259000FD0C88BFBCF5E06F3FF6AFAEB5EB030CAA
:1025A00004BFB6EB020C5FEA500C50F1000041EBA7
:1025B000045170BD0EF0004E4EEA113114EB5C0474
:1025C000C2BFD4EB0C0541EA045170BD41F4801147
:1025D0004FF0000E013C90E645EA060E8DE60CEA4F
:1025E000135594EA0C0F08BF95EA0C0F3FF43BAF6C
:1025F00094EA0C0F0AD150EA01347FF434AF95EA23
:102600000C0F7FF425AF104619462CE795EA0C0F06
:1026100006D152EA03353FF4FDAE1046194622E7D3
:1026200050EA410618BF52EA43067FF4C5AE50EAAD
:1026300041047FF40DAF52EA43057FF4EBAE12E79D
:102640004FEA410212F5001215D211D56FF47873DA
:10265000B3EB625212D94FEAC12343F0004343EA7D
:10266000505311F0004F23FA02F018BF4042704758
:102670004FF00000704750EA013005D111F00040E2
:1026800008BF6FF0004070474FF00000704700BF78
:102690004FEA4102B2F1E04324BFB3F5001CDCF184
:1026A000FE5C0DD901F0004C4FEAC0024CEA5070BC
:1026B000B2F1004F40EB830008BF20F001007047EB
:1026C00011F0804F21D113F13872BCBF01F00040EE
:1026D000704741F480114FEA5252C2F11802C2F120
:1026E000200C10FA0CF320FA02F018BF40F00100A1
:1026F0004FEAC1234FEAD32303FA0CFC40EA0C0053
:1027000023FA02F34FEA4303CCE77FEA625307D18F
:1027100050EA01331EBF4FF0FE4040F440007047C6
:1027200001F0004040F0FE4040F40000704700BF60
:1027300080F0004002E000BF81F0004142001FBF76
:102740005FEA410392EA030F7FEA226C7FEA236C7F
:102750006AD04FEA1262D2EB1363C1BFD218414074
:1027600048404140B8BF5B42192B88BF704710F00A
:10277000004F40F4000020F07F4018BF404211F0AD
:10278000004F41F4000121F07F4118BF494292EA15
:10279000030F3FD0A2F1010241FA03FC10EB0C0041
:1027A000C3F1200301FA03F100F0004302D54942CE
:1027B00060EB4000B0F5000F13D3B0F1807F06D37B
:1027C00040084FEA310102F10102FE2A51D2B1F173
:1027D000004F40EBC25008BF20F0010040EA030068
:1027E0007047490040EB000010F4000FA2F1010215
:1027F000EDD1B0FA80FCACF1080CB2EB0C0200FA9F
:102800000CF0AABF00EBC25052421843BCBFD040EC
:102810001843704792F0000F81F4000106BF80F466
:1028200000000132013BB5E74FEA41037FEA226C29
:1028300018BF7FEA236C21D092EA030F04D092F0F4
:10284000000F08BF0846704790EA010F1CBF002028
:10285000704712F07F4F04D1400028BF40F0004085
:10286000704712F100723CBF00F50000704700F0A5
:10287000004343F0FE4040F4000070477FEA2262CC
:1028800016BF08467FEA23630146420206BF5FEA9D
:10289000412390EA010F40F4800070474FF000039D
:1028A00004E000BF10F0004348BF40425FEA000C64
:1028B00008BF704743F0964301464FF000001CE00C
:1028C00050EA010208BF70474FF000030AE000BF62
:1028D00050EA010208BF704711F0004302D54042A0
:1028E00061EB41015FEA010C02BF84460146002012
:1028F00043F0B64308BFA3F18053A3F50003BCFA2D
:102900008CF2083AA3EBC25310DB01FA02FC6344D9
:1029100000FA02FCC2F12002BCF1004F20FA02F2E0
:1029200043EB020008BF20F00100704702F12002D3
:1029300001FA02FCC2F1200250EA4C0021FA02F234
:1029400043EB020008BF20EADC7070474FF0FF0C39
:102950001CEAD0521EBF1CEAD15392EA0C0F93EA34
:102960000C0F6FD01A4480EA010C400218BF5FEAD6
:1029700041211ED04FF0006343EA501043EA511149
:10298000A0FB01310CF00040B1F5000F3EBF490043
:1029900041EAD3715B0040EA010062F17F02FD2A47
:1029A0001DD8B3F1004F40EBC25008BF20F001002A
:1029B000704790F0000F0CF0004C08BF49024CEA41
:1029C000502040EA51207F3AC2BFD2F1FF0340EAD3
:1029D000C250704740F400004FF00003013A5DDC44
:1029E00012F1190FDCBF00F000407047C2F1000285
:1029F000410021FA02F1C2F1200200FA02FC5FEA72
:102A0000310040F1000053EA4C0308BF20EADC70BB
:102A1000704792F0000F00F0004C02BF400010F42D
:102A2000000F013AF9D040EA0C0093F0000F01F0DA
:102A3000004C02BF490011F4000F013BF9D041EAFC
:102A40000C018FE70CEAD15392EA0C0F18BF93EAFE
:102A50000C0F0AD030F0004C18BF31F0004CD8D128
:102A600080EA010000F00040704790F0000F17BFAF
:102A700090F0004F084691F0000F91F0004F14D0F5
:102A800092EA0C0F01D142020FD193EA0C0F03D14D
:102A90004B0218BF084608D180EA010000F0004050
:102AA00040F0FE4040F40000704740F0FE4040F42B
:102AB000400070474FF0FF0C1CEAD0521EBF1CEACA
:102AC000D15392EA0C0F93EA0C0F69D0A2EB0302E8
:102AD00080EA010C49024FEA402037D04FF0805382
:102AE00043EA111143EA10130CF000408B4238BF47
:102AF0005B0042F17D024FF4000C8B4224BF5B1A55
:102B000040EA0C00B3EB510F24BFA3EB510340EAA2
:102B10005C00B3EB910F24BFA3EB910340EA9C0050
:102B2000B3EBD10F24BFA3EBD10340EADC001B01C0
:102B300018BF5FEA1C1CE0D1FD2A3FF650AF8B4264
:102B400040EBC25008BF20F0010070470CF0004C71
:102B50004CEA50207F32C2BFD2F1FF0340EAC2509C
:102B6000704740F400004FF00003013A37E792F05D
:102B7000000F00F0004C02BF400010F4000F013ABB
:102B8000F9D040EA0C0093F0000F01F0004C02BFB6
:102B9000490011F4000F013BF9D041EA0C0195E71F
:102BA0000CEAD15392EA0C0F08D142027FF47DAFB8
:102BB00093EA0C0F7FF470AF084676E793EA0C0FA8
:102BC00004D14B023FF44CAF08466EE730F0004CA6
:102BD00018BF31F0004CCAD130F000427FF45CAF36
:102BE00031F000437FF43CAF5FE700BF4FF0FF3CA4
:102BF00006E000BF4FF0010C02E000BF4FF0010CF7
:102C00004DF804CD4FEA40024FEA41037FEA226CBF
:102C100018BF7FEA236C11D001B052EA530C18BFE1
:102C200090EA010F58BFB2EB030088BFC81738BF46
:102C30006FEAE17018BF40F0010070477FEA226C34
:102C400002D15FEA402C05D17FEA236CE4D15FEA30
:102C5000412CE1D05DF8040B704700BF8446084664
:102C60006146FFE70FB5FFF7C9FF002848BF10F125
:102C7000000F0FBD4DF808EDFFF7F4FF0CBF01206A
:102C800000205DF808FB00BF4DF808EDFFF7EAFFF4
:102C900034BF012000205DF808FB00BF4DF808EDAF
:102CA000FFF7E0FF94BF012000205DF808FB00BFA4
:102CB0004DF808EDFFF7D2FF94BF012000205DF82A
:102CC00008FB00BF4DF808EDFFF7C8FF34BF012037
:102CD00000205DF808FB00BF42000ED2B2F1FE4FAB
:102CE0000BD34FF09E03B3EB126209D44FEA0023DB
:102CF00043F0004323FA02F070474FF000007047A2
:102D000012F1610F01D1420202D14FF0FF30704742
:102D10004FF00000704700BFFDF707F9002103E006
:102D20000A4B5B584350043109480A4B42189A42F7
:102D3000F6D3094A02E0002313600432074B9A429B
:102D4000F9D300F00DF8804770470000983101007A
:102D500008C0FF1F74C5FF1F00C6FF1F24DAFF1F36
:102D6000224C08B5F5F78DFBF5F7F4FBF5F7A2FD5E
:102D7000F5F7B9FDF5F7B4FCF6F77AF8FCF7E4FDE2
:102D8000F6F7F9FAF5F750FEE08CF5F74DFF2078ED
:102D9000F5F7C0FCE078F5F72DFDF6F745F8218949
:102DA0006079228AFCF794FEF6F736FFF7F71AF9F6
:102DB000FDF75AF80E4B04229A60FBF743F8FBF735
:102DC000E9FC0C4B20229A60FBF734F9FBF732FD4B
:102DD000FBF7E1FCF5F7DCFFF6F716F80028F3D077
:102DE000F7F700F9FBF72EF8EEE700BF0CC0FF1F66
:102DF000C0F00F4000F10F4070B4860746D0541E5B
:102E0000002A41D0CAB2034602E014F1FF343BD39A
:102E100003F8012B9D07F8D1032C2ED9CDB245EA3A
:102E200005250F2C45EA054519D903F11002264660
:102E3000103E0F2E42F8105C42F80C5C42F8085C21
:102E400042F8045C02F11002F2D8A4F1100222F060
:102E50000F0204F00F041032032C13440DD91E4648
:102E60002246043A032A46F8045BFAD8221F22F0CD
:102E700003020432134404F003042CB1C9B21C440D
:102E800003F8011B9C42FBD170BC704714460346FB
:102E9000C2E700BF024B13B1024800F005B870470B
:102EA00000000000B52E0100002301461A46184616
:102EB00000F01EB838B50A4C0A4D641BA4100AD0A5
:102EC00004F18043013B05EB8305013C55F80439CF
:102ED0009847002CF9D1BDE8384000F051B900BF47
:102EE0009831010094310100704700BF704700BF66
:102EF0002DE9F8432C4D0646286898460F46914622
:102F0000FFF7F2FF294B1C68D4F84831002B3ED064
:102F10005A681F2A1CDC02F1010E76B103EB820114
:102F20000124C1F88890D3F8880194402043022EF0
:102F3000C3F88801C1F8088123D00232C3F804E045
:102F4000286843F82270FFF7D1FF0020BDE8F8831E
:102F5000174B0BB34FF4C870AFF300800346D8B1E2
:102F6000D4F848210260002141600A46C4F84801B3
:102F70004FF0010EC0F88811C0F88C11002EDCD083
:102F8000CCE7D3F88C110C43C3F88C41D5E704F59A
:102F9000A673C4F84831BBE72868FFF7A7FF4FF0D6
:102FA000FF30BDE8F88300BF70C5FF1F703101001E
:102FB000000000008025000040380000004B0000A9
:102FC000807000000096000000E10000002C01006D
:102FD00000C201000084030090D0030020A107007C
:102FE00040420F00F4010000640000000180080866
:102FF000000000000064000000000000000000006D
:10300000C80000000000000000000000010003E80C
:103010000000000000000003E800000000000200C3
:10302000FA06000300000000003706000000000060
:10303000000000005AC0FF1F040000000904000047
:1030400098300100A83001000000000000000000DE
:10305000000000000000000031C1FF1FEEC0FF1F94
:103060000000000000000000000000000000000060
:1030700000000000000012004300000000000000FB
:103080000000000003010201100002020010000312
:1030900003011000000100005AC0FF1FB4C0FF1F51
:1030A0008EC0FF1F6CC0FF1F043A2622151C0100B2
:1030B00011050100A9050100190301003D170100D8
:1030C0003D1701003D1701003D1701003D170100AC
:1030D0003D1701003D1701003D1701003D1701009C
:1030E0003D1701003D1701003D1701009B0801003D
:1030F00031080100910801005D080100310801005C
:103100003D1701001D08010009090100D91901003E
:10311000A51A010000000000A51A0100000000002F
:1031200099190100C11901000000000001190100F6
:1031300031190100991B0100791B0100D51801000C
:103140000101000101000000000101000000000079
:103150000101010101000000010100010100010065
:1031600000010000010000313131305631313100B1
:1031700048C1FF1FF8B500BFF8BC08BC9E467047A9
:0C318000F8B500BFF8BC08BC9E467047C4
:08318C00952E010035840000BE
:0431940011840000A2
:103198006731010000010200000800000100000082
:1031A8000200000000000000000000000000000015
:1031B8000000000000000000000007000000000000
:1031C80000000000000000000000000000000000F7
:1031D80000000000040506A1200000000002000015
:1031E80000FF0403090400C20100000008000000F9
:1031F8000000000022034200410044002000530068
:103208005400520049004E004700200049004E007B
:103218004400450058002603530074006500700000
:1032280070006500720020004D006F0074006F0090
:103238007200200044006500760020003A03540024
:10324800520049004E0041004D0049004300200053
:103258004D006F00740069006F006E00200043008D
:103268006F006E00740072006F006C002000200078
:1032780020002000200009024300020100C032099A
:1032880004000001020200000524001001052401C9
:103298000101042402060524060001070583031022
:1032A800000A09040100020A000000070581021053
:1032B80000000705020210000012010002020000CF
:1032C800103C2A0001020001020001000000000079
:1032D8000000000034C4FF1F9CC4FF1F04C5FF1F6B
:1032E80000000000000000000000000000000000D6
:1032F80000000000000000000000000000000000C6
:1033080000000000000000000000000000000000B5
:1033180000000000000000000000000000000000A5
:103328000000000000000000000000000000000095
:103338000000000000000000000000000000000085
:103348000000000000000000000000000000000075
:103358000000000000000000000000000000000065
:103368000000000000000000000000000000000055
:103378000000000000000000010000000000000044
:103388000E33CDAB34126DE6ECDE05000B00000009
:103398000000000000000000000000000000000025
:1033A8000000000000000000000000000000000015
:1033B8000000000000000000000000000000000005
:1033C80000000000000000000000000000000000F5
:0C36F800000000000000000000DAFF1FCE
:103704009831010008C0FF1F6C0500000000000094
:083714000000000000000000AD
:0400000310002D19A3
:00000001FF
